:020000040000fa
:080000000002040000000000f2
:020000040000fa
:04000800cc03000025
:020000040000fa
:04000c00e403000009
:020000040000fa
:04001000fc030000ed
:020000040000fa
:04001400d403000011
:020000040000fa
:04001800ec030000f5
:020000040000fa
:04001c00f4030000e9
:020000040000fa
:0400200004040000d4
:020000040000fa
:040024008e04000046
:020000040000fa
:04002800940400003c
:020000040000fa
:04002c009404000038
:020000040000fa
:040030009404000034
:020000040000fa
:040034009404000030
:020000040000fa
:04003800940400002c
:020000040000fa
:04003c009404000028
:020000040000fa
:040040009404000024
:020000040000fa
:04004400a203000013
:020000040000fa
:04004800940400001c
:020000040000fa
:04004c009404000018
:020000040000fa
:040050009404000014
:020000040000fa
:040054009404000010
:020000040000fa
:04005800940400000c
:020000040000fa
:04005c001c04000080
:020000040000fa
:040060009404000004
:020000040000fa
:040064009404000000
:020000040000fa
:0400680094040000fc
:020000040000fa
:04006c0094040000f8
:020000040000fa
:0400700094040000f4
:020000040000fa
:0400740094040000f0
:020000040000fa
:0400780094040000ec
:020000040000fa
:04007c0094040000e8
:020000040000fa
:0400800094040000e4
:020000040000fa
:0400840094040000e0
:020000040000fa
:0400880094040000dc
:020000040000fa
:04008c0094040000d8
:020000040000fa
:0400900094040000d4
:020000040000fa
:0400940094040000d0
:020000040000fa
:0400980094040000cc
:020000040000fa
:04009c0094040000c8
:020000040000fa
:0400a00094040000c4
:020000040000fa
:0400a40094040000c0
:020000040000fa
:0400a80094040000bc
:020000040000fa
:0400ac0094040000b8
:020000040000fa
:0400b00094040000b4
:020000040000fa
:0400b40094040000b0
:020000040000fa
:0400b80094040000ac
:020000040000fa
:0400bc0094040000a8
:020000040000fa
:0400c00094040000a4
:020000040000fa
:0400c40094040000a0
:020000040000fa
:0400c800940400009c
:020000040000fa
:0400cc009404000098
:020000040000fa
:0400d0009404000094
:020000040000fa
:0400d4009404000090
:020000040000fa
:0400d800940400008c
:020000040000fa
:0400dc009404000088
:020000040000fa
:0400e0009404000084
:020000040000fa
:0400e4009404000080
:020000040000fa
:0400e800940400007c
:020000040000fa
:0400ec009404000078
:020000040000fa
:0400f0009404000074
:020000040000fa
:0400f4009404000070
:020000040000fa
:0400f800940400006c
:020000040000fa
:0400fc009404000068
:020000040000fa
:040100009404000063
:020000040000fa
:04010400940400005f
:020000040000fa
:04010800940400005b
:020000040000fa
:04010c00820300006a
:020000040000fa
:040110009404000053
:020000040000fa
:04011400940400004f
:020000040000fa
:04011800940400004b
:020000040000fa
:04011c009404000047
:020000040000fa
:040120009404000043
:020000040000fa
:04012400940400003f
:020000040000fa
:04012800940400003b
:020000040000fa
:04012c009404000037
:020000040000fa
:040130009404000033
:020000040000fa
:04013400940400002f
:020000040000fa
:04013800940400002b
:020000040000fa
:04013c009404000027
:020000040000fa
:040140009404000023
:020000040000fa
:04014400940400001f
:020000040000fa
:04014800940400001b
:020000040000fa
:04014c009404000017
:020000040000fa
:040150009404000013
:020000040000fa
:04015400940400000f
:020000040000fa
:04015800940400000b
:020000040000fa
:04015c009404000007
:020000040000fa
:040160009404000003
:020000040000fa
:0401640094040000ff
:020000040000fa
:0401680094040000fb
:020000040000fa
:04016c0094040000f7
:020000040000fa
:0401700094040000f3
:020000040000fa
:0401740094040000ef
:020000040000fa
:0401780094040000eb
:020000040000fa
:04017c0094040000e7
:020000040000fa
:0401800094040000e3
:020000040000fa
:0401840094040000df
:020000040000fa
:0401880094040000db
:020000040000fa
:04018c0094040000d7
:020000040000fa
:0401900094040000d3
:020000040000fa
:0401940094040000cf
:020000040000fa
:0401980094040000cb
:020000040000fa
:04019c0094040000c7
:020000040000fa
:0401a00094040000c3
:020000040000fa
:0401a40094040000bf
:020000040000fa
:0401a80094040000bb
:020000040000fa
:0401ac0094040000b7
:020000040000fa
:0401b00094040000b3
:020000040000fa
:0401b40094040000af
:020000040000fa
:0401b80094040000ab
:020000040000fa
:0401bc0094040000a7
:020000040000fa
:0401c00094040000a3
:020000040000fa
:0401c400940400009f
:020000040000fa
:0401c800940400009b
:020000040000fa
:0401cc009404000097
:020000040000fa
:0401d0009404000093
:020000040000fa
:0401d400940400008f
:020000040000fa
:0401d800940400008b
:020000040000fa
:0401dc009404000087
:020000040000fa
:0401e0009404000083
:020000040000fa
:0401e400940400007f
:020000040000fa
:0401e800940400007b
:020000040000fa
:0401ec009404000077
:020000040000fa
:0401f0009404000073
:020000040000fa
:0401f400940400006f
:020000040000fa
:0401f800940400006b
:020000040000fa
:0401fc009404000067
:020000040000fa
:040200009404000062
:020000040000fa
:04020400940400005e
:020000040000fa
:04020800940400005a
:020000040000fa
:04020c009404000056
:020000040000fa
:040210009404000052
:020000040000fa
:04021400940400004e
:020000040000fa
:04021800940400004a
:020000040000fa
:04021c009404000046
:020000040000fa
:040220009404000042
:020000040000fa
:04022400940400003e
:020000040000fa
:04022800940400003a
:020000040000fa
:04022c009404000036
:020000040000fa
:040230009404000032
:020000040000fa
:04023400940400002e
:020000040000fa
:04023800940400002a
:020000040000fa
:04023c009404000026
:020000040000fa
:040240009404000022
:020000040000fa
:04024400940400001e
:020000040000fa
:04024800940400001a
:020000040000fa
:04024c009404000016
:020000040000fa
:040250009404000012
:020000040000fa
:04025400940400000e
:020000040000fa
:04025800940400000a
:020000040000fa
:04025c009404000006
:020000040000fa
:040260009404000002
:020000040000fa
:0402640094040000fe
:020000040000fa
:0402680094040000fa
:020000040000fa
:04026c0094040000f6
:020000040000fa
:0402700094040000f2
:020000040000fa
:0402740094040000ee
:020000040000fa
:0402780094040000ea
:020000040000fa
:04027c0094040000e6
:020000040000fa
:0402800094040000e2
:020000040000fa
:10040000cfa122000eff27000e018800000000008f
:10041000000020000000e000020032000001200087
:100420002002880014000700440107000000e000db
:1004300003003a00c03c2300010020000200370006
:100440000000200001002000810f70000100320038
:100450000f000700000020000000e0000200320052
:100460000000020000000000ce4c0200000000006e
:100470000040da000000fe00400320000000e00021
:1004800002003200002020009001880000000600d9
:10049000a1028800800478000000eb001f003700f4
:1004a000e284440054a0b4009905ba00e2844400f8
:1004b00054a0b4009906ba00e284440054a0b400e9
:1004c0000006eb00476fde00fd07b200ae018800ba
:1004d000636ce10003003a000ad801000000eb0061
:1004e0000e003700606ce10008003a00004deb00a0
:1004f0000a05e800020039003420ec000af0a000f0
:100500008b05e900f9ff3e00040037006168e10057
:10051000010032000086eb000b00070019c7ba008b
:100520000e04e0001905ba0003003a000a00e000da
:10053000dbff3a0000000600fe07b200ae028800b2
:100540008a047800f5ff37000cd0a300e20f4d00bd
:100550001c00390089027800354dba000a05e80010
:10056000020039003420ec000af0a0008b05e900fd
:100570000f003200254dba000a05e80002003900dc
:100580003420ec000af0a0008b05e90008003200de
:100590000c00e0000600320015cdba000a05e800a4
:1005a000020039003420ec000af0a0008b05e900bd
:1005b0008984e80054a0b4000b00e000e2ff3a0098
:1005c000000006009902ba00055d78008b05e9007d
:1005d000f7ff3200c82ade00055d78008b05e900d0
:1005e000f3ff32000c00e000f1ff320019ddba0029
:1005f000eeff3700664d040000000000684d040067
:10060000000000006a4d040000000000424d04009c
:1006100000000000464d0400000000004a4d0400a8
:10062000000000004e4d0400000000001a410400cc
:1006300000000000204104000000000024410400ec
:100640000000000028410400000000007c2d040090
:1006500000000000862c040000000000f82c0400bc
:1006600000000000462e040000000000b22104003b
:1006700000000000a821040000000000024904005e
:1006800000000000044904000000000006490400c6
:100690000000000008490400000000000a490400ae
:1006a000000000000c49040000000000361c04009b
:1006b00000000000441c0400000000005a21040057
:1006c00000000000ba20040000000000721e0400b8
:1006d00000000000dc1f0400000000004c0a0400c1
:1006e00000000000d009040000000000980d040084
:1006f000000000004c0e040000000000261604005c
:10070000000000003600f800809fbe00829fbe00ff
:10071000849fbe00869fbe00e08e80000000e00047
:1007200001003200000001000728a9004f03be00ad
:100730004f02be004f01be004f00be003600f90060
:10074000004006003600f800809fbe00829fbe0079
:10075000849fbe00869fbe00f08e80000000e000f7
:100760000100320000000100f07f22001048e80084
:1007700011c0b3000000e9000148780000e8a900ba
:100780004f03be004f02be004f01be004f00be002f
:100790003600f900004006003600f800c028a90025
:1007a0000000eb00b12407003600f800e07d2200d5
:1007b000800778007800400000018800c048a90048
:1007c00010002000a92407003600f800c068a90026
:1007d00020002000a52407003600f800c088a900ea
:1007e00030002000a12407003600f800c0a8a900ae
:1007f000400020009d2407003600f800c608a9002c
:1008000070002000992407003600f800c4a8ab004f
:1008100003003200c4a8a900900020009324070020
:10082000c488ab0003003200c488a900a0002000e7
:100830008e240700ffff37003600f800809fbe00bf
:10084000829fbe00849fbe00869fbe00881f7800e6
:100850003200f8003400f80010002000a0018800e9
:10086000002020009001880000000000350ea80044
:1008700080240700c03b890000512200f4080700d3
:1008800001a8a9008067220050240700207c2200d4
:100890005224070060742200b11f0700f07022008c
:1008a000e411e30002003e00e431ec000060fe00d1
:1008b000d13e8100601a2d00808f500005003a0063
:1008c000c03e81000018a3000200320000000000ba
:1008d000feff37006724070088772200ee004400ff
:1008e000980850007124070062240700f0004400bb
:1008f00098085000350ea9003400f9003200f900c4
:100900004f0478004f03be004f02be004f01be00ef
:100910004f00be003600f900004006003600f80027
:1009200080002000672407003600f800c8c8bf0018
:100930000080fb000010b0006224070000000500ea
:100940008f1fd1000f0007008f87e9000000e00033
:1009500000000600809feb000a0007008f87e90077
:100960000000e000000006001400200040003700f6
:10097000f4ff2f003e003700600007000400be00b7
:1009800000000600889fbe008a9fbe008c9fbe00ac
:100990000404be000605be00809fbe00829fbe000c
:1009a00021000700040678000800be000a01be000e
:1009b0001d000700840678004f03be004f02be00f2
:1009c0008d4f76007fb0970013003300f0ff2f00ab
:1009d0008b8f6b0006003b000d0666000c00a70025
:1009e0000a00370007f0a600100020000a003700b8
:1009f000880f5200898f5a008a0f5b008b8f5b0033
:100a0000030039001000200001003e00000020001b
:100a100007f0a7000000ea004f06be004f05be0029
:100a20004f04be000000060005ff2700058261009c
:100a3000070032000428e100010032002400050014
:100a40000600070001003a00440005000408050004
:100a500002000700f9ff3a00140005006f826100f0
:100a6000810270008502710085027200000006009c
:100a7000889fbe008a9fbe00841f78001700070071
:100a80004f00780011003300f0ff2f00838f6c00bf
:100a900006003b00040565000a00a70008003700b7
:100aa00009f0a6001000200008003700820f540053
:100ab000838f5c00030039001000200001003e001d
:100ac0000000200009f0a7000000ea004f05be006a
:100ad0004f04be000000e000000006000004be005d
:100ae000160007000003be000405be000200be00a1
:100af00012000700844f7500000006006022b80055
:100b0000060220000000d0008180d2000482d200c2
:100b10008582d2000000a0000202520083825a00a7
:100b2000030031000202420083824a000000a1005b
:100b30000603e900f3ff3a0000000600c70ade00e2
:100b4000f107b200f50fb20008003200e1cf420019
:100b5000020032000170a00024000500810f700027
:100b6000010032000408050044000500810f7000f8
:100b700002003a00140005008502e9000000400070
:100b800081c04800fcff3b000170a000240005006c
:020000040000fa
:100b9000ffff00004c0a0000d0090000980d000083
:100ba0004c0e0000261600000000000000000000af
:100bb0000000000000000000000000000000000035
:100bc000010000001c1100000000000000000000f7
:100bd000446500006320000031380000203200002e
:100be0003031000039310000303a00003334000069
:080bf0003a3100003200000060
:020000040000fa
:100bf8001800fa00889fbe008a9fbe008c1f7800ec
:100c080000067800f4af9f0085b79f0096b79f0055
:100c1800a7b79f002c709000ef4060000068a30009
:100c28000b003200e4cf50003b003200e8cf500008
:100c38004e0032000046eb000c4078004f0678006a
:100c48004f05be004f04be000080fa0000000600f9
:100c58000058a30018003200e2cf500067003200ad
:100c68008c003e00e1cf5000f2ff3a008c69900002
:100c78000c6090006fda97003c299000e10f51005a
:100c8800250132000046eb0080cf5100eaff340016
:100c980001467800844f5000e6ff35000c4078008c
:100ca8004f0678004f05be004f04be000080fa00d2
:100cb80000000600e6ff3700e2cf50006200320075
:100cc800a6003e00e1cf5000daff3a008c699000a0
:100cd8000c6090006fda97003c299000e10f5100fa
:100ce800000132000046eb0080cf5100d2ff3600f1
:100cf80001467800844f5000ceff39000c40780040
:100d08004f0678004f05be004f04be000080fa0071
:100d180000000600ceff37004c109000dc10900059
:100d28000c1490009c1490007fad97008fb597002d
:100d38003c2e9000e10f5600870132000801be00ea
:100d480009ff07000000e000baff34001cc0b30030
:100d58000801be000a00be0001ff07000000e00015
:100d6800b5ff34000046eb00b3ff37004c1090008d
:100d7800dc1090006c119000fc1190000c14900095
:100d88009c1490002c159000bc1590007faa970029
:100d98008fb297001fb39700afb39700b4b79f0007
:100da800c5b79f00d6b79f00e7b79f003c2e9000bd
:100db800e10f5600530132000802be000a03be00cc
:100dc800e2fe07000000e0009aff34001cc0b300f8
:100dd8000802be000a03be003fb09700cfb09700dc
:100de8005fb19700efb19700d3fe07000000e00065
:100df80091ff34000046eb008fff37004c11900044
:100e08000c109000ffa99700bc289000e18f5000bb
:100e1800db0032000046eb00800f510086ff3400f3
:100e28001cc0b300830f500082ff35000c407800cf
:100e38004f0678004f05be004f04be000080fa0040
:100e48000000060082ff37004c1190000c10900043
:100e5800ffa99700bc289000e18f5000bb0032002a
:100e68000046eb00800f510073ff36001cc0b30032
:100e7800830f50006fff39000c4078004f06780050
:100e88004f05be004f04be000080fa0000000600b7
:100e98006fff3700e4cf50007a003200e8cf5000ef
:100ea80064ff3a004c149000dc1490006c1590001c
:100eb800fc159000f8b79f0089bf9f009abf9f005c
:100ec800abbf9f000c1090009c1090002c1190005c
:100ed800bc119000b4b79f00c5b79f00d6b79f005c
:100ee800e7b79f00bc2a9000e18f5200ea00320069
:100ef8000046eb007fb497008fbc97001fbd97009a
:100f0800afbd97000040e10001c8e10002d0e10058
:100f180003d8e10048ff34001cc0b3003fb297007b
:100f2800cfb297005fb39700efb397000400e100da
:100f38000588e1000690e1000798e1003dff3500d3
:100f48000c4078004f0678004f05be004f04be00e5
:100f58000080fa00000006003dff3700e4cf500093
:100f680030003200e8cf500032ff3a004c149000b5
:100f7800dc1490006c159000fc159000f8b79f00e9
:100f880089bf9f009abf9f00abbf9f000c109000c5
:100f98009c1090002c119000bc119000b4b79f00d9
:100fa800c5b79f00d6b79f00e7b79f00bc2a90003f
:100fb800e18f52009d0032000046eb007fb497009d
:100fc8008fbc97001fbd9700afbd97000040e100a0
:100fd80001c8e10002d0e10003d8e10016ff3600a5
:100fe8001cc0b3003fb29700cfb297005fb3970021
:100ff800efb397000400e1000588e1000690e100e6
:101008000798e1000bff39000c4078004f06780084
:101018004f05be004f04be000080fa000000060025
:101028000bff37004c129000dc1290000c1090005f
:101038009c1090007fab97008fb397003c299000dd
:10104800e10f51006a0032000046eb00800f5200a9
:10105800818f5a00f8fe36001cc0b300860f50007e
:10106800878f5800f3fe39000c4078004f0678004f
:101078004f05be004f04be000080fa0000000600c5
:10108800f3fe37004c129000dc1290000c10900018
:101098009c1090007fab97008fb397003c2990007d
:1010a800e10f5100430032000046eb00800f520070
:1010b800818f5a00e0fe34001cc0b300860f500038
:1010c800878f5800dbfe35000c4078004f0678000b
:1010d8004f05be004f04be000080fa000000060065
:1010e800dbfe37000046eb0080cf5100d2fe310016
:1010f80002467800844f5000cefe3e000c40780037
:101108004f0678004f05be004f04be000080fa006d
:1011180000000600cefe37000046eb0080cf5100ed
:10112800c5fe3d0002467800844f5000c1fe3c00d9
:101138000c4078004f0678004f05be004f04be00f3
:101148000080fa0000000600c1fe37000046eb00f0
:10115800800f5100b8fe310001467800830f50001f
:10116800b4fe3e000c4078004f0678004f05be00e4
:101178004f04be000080fa0000000600b4fe3700ed
:101188000046eb00800f5100abfe3d0001467800a1
:10119800830f5000a7fe3c000c4078004f067800f3
:1011a8004f05be004f04be000080fa000000060094
:1011b800a7fe37000046eb00800f5200818f5a00cf
:1011c8009dfe3d0002467800860f5000878f58002c
:1011d80098fe3c000c4078004f0678004f05be0092
:1011e8004f04be000080fa000000060098fe370099
:1011f8000046eb00800f5200818f5a008efe3100ae
:1012080002467800860f5000878f580089fe3e00fe
:101218000c4078004f0678004f05be004f04be0012
:101228000080fa000000060089fe37000046eb0047
:101238007fb497008fbc97001fbd9700afbd970084
:101248000040e10001c8e10002d0e10003d8e1005c
:1012580079fe3100054678003fb29700cfb297007b
:101268005fb39700efb397000400e1000588e10041
:101278000690e1000798e1006efe3e000c40780001
:101288004f0678004f05be004f04be000080fa00ec
:10129800000006006efe37000046eb007fb49700a2
:1012a8008fbc97001fbd9700afbd97000040e100bd
:1012b80001c8e10002d0e10003d8e1005efe3d0074
:1012c800054678003fb29700cfb297005fb397000a
:1012d800efb397000400e1000588e1000690e10003
:1012e8000798e10053fe3c000c4078004f06780058
:1012f8004f05be004f04be000080fa000000060043
:1013080053fe37000802be000a03be008afd07002c
:101318000000e00047fe3d000802be000a03be00d0
:101328003fb09700cfb097005fb19700efb197003b
:1013380086fd07000000e0003efe35000c40780006
:101348004f0678004f05be004f04be000080fa002b
:10135800000006003efe37000801be0080fd0700c1
:101368000000e00033fe3d000801be000a00be0098
:101378007dfd07000000e0002efe35000c407800df
:101388004f0678004f05be004f04be000080fa00eb
:10139800000006002efe3700889fbe008a9fbe0010
:1013a8000088eb008001eb00130098000042eb007e
:1013b8002350980023009800345098003300980078
:1013c80044509800430098005450980053009800e7
:1013d8006450980063009800745098007300980057
:1013e8000458980003089800145898005108980069
:1013f8006044b8006055b8000810980019109800ab
:101408002a1098003b10980048109800591098002e
:101418006a1098007b1098000318980024709800b0
:10142800231898006033b8003618980047189800b9
:1014380024789800347898006318980073189800f6
:101448000320980024c09800262098003720980090
:10145800462098005720980044c8980076209800a5
:1014680007289800122898002328980011002000c7
:10147800312898006208980073089800418f80000e
:10148800c00898004f05be004f04be0000000600cb
:101498000800fa00889fbe008a9fbe008c1f780053
:1014a800000678002c189000e60f500019003e0046
:1014b800e50f5000370039008c1890002c70900010
:1014c8006f406000e24f50008b01320034013e0053
:1014d800e14f5000550132007fb297008fba970054
:1014e8001fbb9700afbb97000c007800c0fd07003a
:1014f8000004e0001c01320040002000201e98007b
:101508004f0678004f05be004f04be000080fa0069
:1015180000000600e70f500085003200e80f500079
:10152800f7ff3a007c189000ec1890000001e800e2
:10153800721e9800810f5000f1ff39000000eb0087
:10154800701e98002c7890000080fb008000eb0053
:101558004c219000dc21900000004100818049006e
:101568004026980051269800e00f5000e08f580060
:10157800e3ff350020002000201e98004f06780069
:101588004f05be004f04be000080fa0000000600b0
:10159800e0ff3700e20f5000a6003200e40f5000d1
:1015a800db003200e10f5000d5ff3a007c189000b4
:1015b800ec1890000001e800721e9800810f50009e
:1015c8002e0039000000eb00701e98003c199000b6
:1015d800cc1990002c7a90000482fb008002eb006a
:1015e80004024100858249006c089000fc089000c4
:1015f800800f5200818f5a00030036006011b80036
:10160800321e9800431e98008043eb008782fb003f
:101618000040eb000503e800f282420006034300a5
:101628000603460085024600dc08900082804000e0
:101638000082fb00160242009448780061014100d4
:10164800e0814900321e9800431e98000040e800df
:10165800954f5000f4ff39008743e8003c7890002c
:1016680080cf5300e9ff39007c2090008c2890003f
:10167800820f5000838f5800e90036008c189000c4
:101688002c7090006f406000e24f50002201320041
:10169800d0003e00e14f5000f90032000802be00c1
:1016a8000a03be000c00780051fd07000004e000aa
:1016b800a30032004cc890000004e000a0003200f3
:1016c8002c209000bc209000e00f5000e08f5800c4
:1016d800f00035003c189000cc189000e00f500046
:1016e800e08f5800f80032007c1990000200e000fa
:1016f800fc003a002c7990000281fb008001eb008d
:101708000200500083805800402698005126980017
:1017180070002000201e98004f0678004f05be007c
:101728004f04be000080fa000000060079ff370071
:101738007c189000ec1890000001e800721e9800d8
:10174800810f50006eff39000000eb00701e9800fa
:101758003c199000cc1990002c7a90000482fb0070
:101768008002eb0004024100858249006c08900069
:10177800fc089000800f5200818f5a000400360048
:101788006033b800361e9800471e98006011b800f4
:101798008043eb008782fb000040eb000503e80074
:1017a800f282420006034300060346008502460013
:1017b800dc089000828040000082fb001602420094
:1017c8009448780061014100e0814900321e980088
:1017d800431e98000040e800954f5000f4ff390080
:1017e8008743e8003c78900080cf5300e9ff390038
:1017f8004c209000dc2090000201500083815800aa
:101808002c209000bc209000800f5100818f59003f
:1018180079003e000000eb00201e98004f0678007b
:101828004f05be004f04be000080fa00000006000d
:1018380038ff37007c189000ec1890000001e80091
:10184800721e9800810f5000280039000000eb003c
:10185800701e98003c199000cc1990008043eb0052
:101868008782fb000040eb000503e800f28242009b
:10187800060343000603460085024600dc08900084
:10188800828040000082fb001602420094487800e3
:1018980061014100e0814900321e9800431e980012
:1018a8000040e800954f5000f4ff39008743e800f6
:1018b8003c78900080cf5300e9ff39002c789000e5
:1018c8000080fb008000eb0002014000838148009b
:1018d8006c089000fc089000800f5100818f59001f
:1018e800020036000000eb00201e98000c2090003b
:1018f8000000e800002698004f0678004f05be005b
:101908004f04be000080fa000000060001ff370007
:101918000c2090000000e800002698007c18900039
:101928000000e800701e98004f0678004f05be00c2
:101938004f04be000080fa0000000600f5fe3700e4
:1019480048169800591698006a1698007b16980051
:101958004f0678004f05be004f04be000080fa0015
:1019680000000600ebfe37007fb097008fb89700a5
:101978001fb99700afb99700401698005116980004
:1019880062169800731698004f0678004f05be003f
:101998004f04be000080fa0000000600ddfe37009c
:1019a800e44f50002a003200e84f5000cafe3a00c7
:1019b800110278009102900021039000b103900079
:1019c800f4b79f0085bf9f0096bf9f00a7bf9f00e9
:1019d800c1fe3700e44f500025003200e84f5000a8
:1019e8002eff3a0011047800910490002105900020
:1019f800b105900029ff37001c2a9000ac2a9000fe
:101a08000201420083814a00820f5000838f5800f0
:101a1800bbfe39000000eb00201e98007fff370056
:101a280010c0b30040ce980014ff37001140780072
:101a38000082fb008002eb006033b800f4b79f001f
:101a480085bf9f0096bf9f00a7bf9f00a2fe3700db
:101a580011027800910290006033b800f4b79f003b
:101a680085bf9f0096bf9f00a7bf9f009afe3700c3
:101a780011047800910490006055b80007ff370002
:101a8800114478000884fb008004eb006055b8001e
:101a980002ff370040269800512698006022b800bf
:101aa800341e9800451e980080002000201e9800d3
:101ab8004f0678004f05be004f04be000080fa00b4
:101ac8000000060093fe37002c7890000080fb0091
:101ad8008000eb001c299000ac2990000000510008
:101ae80081805900402698005126980070002000f7
:101af800201e980008ff3700110078006102b80026
:101b08006033b800f4b79f0085bf9f0096bf9f0061
:101b1800a7bf9f0070fe3700110478008004eb0017
:101b28006055b800ddfe37004071900082487800ab
:101b3800307a90009440980040799000a240980034
:101b4800507a9000b440980060719000c2409800ac
:101b580030199000c0199000481add004811de00c5
:101b680002017200c819de00d24098000079900086
:101b7800e2409800107a9000f440980020599000b4
:101b88008248980050099000cf91de00481add0085
:101b98004811de0002017200c819de009248980060
:101ba80050099000cf91de00a3489800500990009a
:101bb800cf91de004819de00b248980040c190007d
:101bc800c248980020219000b0219000481add00fa
:101bd8004811de0002017200d248980060c19000ee
:101be800e248980070c29000f448980000c990003c
:101bf8008250980040219000d0219000481add00c2
:101c08004811de00020172009250980020c990002d
:101c1800a250980030ca9000b450980020d190008b
:101c2800c250980010299000a0299000481add00a1
:101c38004811de0002017200c819de00d250980077
:101c480040d19000e250980050d29000f450980093
:101c5800405990008258980060099000f00990005f
:101c6800481add004811de0002017200c819de00c2
:101c78009258980060599000a258980070589000a7
:101c8800b058980020c8b300c0589800d00105008b
:101c98006f02b000889fbe008a9fbe008c9fbe0066
:101ca8008e1f78000004be00824678001ac0b30078
:101cb800e3cf5600c5003600090678005c4078007e
:101cc800e84f5000c1003e000004e000bf003200b1
:101cd8008000eb00211c98000040eb00317c98004c
:101ce800012498006011b800321c9800431c980029
:101cf800394190004811dd00a94090008180fb0027
:101d080081004100611c9800711c98006022b80095
:101d18006033b8004414980055149800661498006d
:101d280077149800207c980021c0b30021c4980043
:101d380040cc98006022b8004424980055249800ac
:101d48001c04e000aa0232004ac0b30080457800b3
:101d58000c077800ede79f000a46e8000a80fb00c0
:101d68000080440010407800e14f5000df0032004e
:101d78009d0031008b86fb000c86fb000d00e800ff
:101d880000004000000044000c8644008c00e8007d
:101d98001181fb008001eb00481add00c812de004b
:101da800850272004812dd001c81fb008001eb00f7
:101db800020842004c4090008d064400a05698004e
:101dc8002879900002414000227c9800a8c0900029
:101dd80000c0400020c49800680e9000f80e9000e3
:101de8000281fb008001eb000c00be00e0fa070056
:101df8000000560081805e00102c9800212c98006d
:101e0800664545008b45e8009ecf1500d2ff3e0091
:101e18000e067800efe697008a80fb000a45e80086
:101e28000a80fb008a45e8008180440091407800e0
:101e3800e1ef9f0021749800008044001040780072
:101e4800e14f50008a023200760131000b82fb001c
:101e5800048244000400e8001081fb008001eb00cc
:101e6800481bdd00c813de00870373004813dd003c
:101e78000480e8001081fb008001eb00c011dd0048
:101e88000200200006034100878349001481fb00fb
:101e98008001eb000601410087814900021c98007f
:101ea8006feb970064c74500ef456300e2cf55002c
:101eb8008d023200a4013e00e1cf55004e003a00e9
:101ec8008e81fb0083814400134278000482fb006a
:101ed8008002eb006033b8000414980015149800d1
:101ee8002614980037149800efea97000504e000dc
:101ef80093013500854078000154a00021749800b2
:101f0800644547008a80fb00818044000100e800a6
:101f18001081fb008001eb00481add00c812de00ca
:101f2800850272004812dd000180e8001081fb0084
:101f38008001eb00c011dd00020020000401410017
:101f4800858149001182fb008002eb0002014200fa
:101f580083814a00e38040001180fb008000eb0091
:101f6800c800dd0000002000020040008380480017
:101f780020249800312498008015070070249800c8
:101f8800012c9800644045000080fb00008044005c
:101f98001080fb00302c9800654545008acf56001c
:101fa800400136000a80fb000080440016c0b300e0
:101fb800904f1300720032001c4678003c7c980059
:101fc8001980fb00201c98000045eb000a407800af
:101fd8004f0778004f06be004f05be004f04be00f5
:101fe8006f02b10000000600e24f500025003200e9
:101ff800e34f5000090032001ac0b3000a407800cd
:102008004f0778004f06be004f05be004f04be00c4
:102018006f02b10000000600f3ff37000c86fb00da
:102028000c864400ac409000bc419000408f80007a
:10203800100178000200e000efff3200c819dd004f
:102048008180fb008181410092007800818f5100de
:10205800720032000100e000e7ff32006400410036
:102068000001780090007800818f51006b003200e9
:10207800640040000100e000f9ff3a001ac0b30014
:10208800deff37000c86fb000c864400ac40900055
:10209800bc419000408f8000100178000200e000f1
:1020a800d5ff3200c819dd008180fb008181410025
:1020b80092007800818f5100b80032000100e000e2
:1020c800cdff3200640041000001780090007800e4
:1020d800818f5100b1003200640040000100e0002f
:1020e800f9ff3a001ac0b300c4ff37000c86fb00a2
:1020f8000c8644008c007800b141780011427800c9
:10210800ac4090003c439000428f800092027800df
:102118000500e00008003a00004078004f0778000a
:102128004f06be004f05be004f04be006f02b1004f
:1021380000000600acff37004833dd008180fb005b
:102148000103430095007800810f530055003200c9
:102158000100e000f0ff3200648042008002780055
:1021680090007800810f53004e0032006400400058
:102178000100e000f9ff3a001ac0b3009fff3700e2
:1021880088189000287090006f406000e24f50005f
:102198008c02320076023e00864f50000e0032005c
:1021a8007fa097008fa897001fa99700afa9970055
:1021b8004014980051149800621498007314980001
:1021c8001c4678003c7c98001980fb00201c980075
:1021d8000045eb007dff3700114078000082fb00ce
:1021e8008002eb006033b800f4a79f0085af9f0022
:1021f80096af9f00a7af9f007fa097008fa897007a
:102208001fa99700afa9970040149800511498008f
:102218006214980073149800e9ff37000100e00089
:1022280075ff3200920090000100e00072ff32005a
:102238008b86fb000d00e800000040000000440011
:10224800110878004c4090008d064400a056980074
:102258002879900002414000227c9800a8c0900094
:1022680000c0400020c49800680e9000f80e90004e
:102278000281fb008001eb000c00be00bcf90700e6
:102288000000560081805e00102c9800212c9800d8
:10229800664545008b45e8009ecf1500aefe3e0022
:1022a800dbfe37000100e00053ff3200150090000c
:1022b8000000e00050ff3200100378009202900006
:1022c80015017800820f53000c0032000200e00074
:1022d80049ff3200ec804200810278001101780049
:1022e800820f530005003200ec8040000200e0003d
:1022f800f9ff3a001ac0b30040ff37000200e000bf
:102308003dff32000500e0003bff32008b86fb00fa
:10231800c820dd008381fb008380400055019000c8
:10232800020001008d00e800818040008100440027
:10233800800878000000e0002fff32004c40900039
:102348008d064400a056980028799000024140006c
:10235800227c9800a8c0900000c0400020c49800cb
:10236800680e9000f80e90000281fb008001eb00df
:102378000c00be007ef907000000560081805e0058
:10238800102c9800212c9800664545008b45e800e4
:102398009ecf150070fe3e009dfe37000100e00054
:1023a80015ff3200920090000100e00012ff320099
:1023b8008b86fb000d00e800000040000000440090
:1023c800010878004c4090008d064400a056980003
:1023d8002879900002414000227c9800a8c0900013
:1023e80000c0400020c49800680e9000f80e9000cd
:1023f8000281fb008001eb000c00be005cf90700c5
:102408000000560081805e00102c9800212c980056
:10241800664545008b45e8009ecf15004efe3e0000
:102428007bfe3700e24f5000f5003200e34f5000ca
:10243800f1fe3a000b80fb0000804400204290002f
:1024480030419000408f8000900178001ac0b3009e
:102458000300e000ddfe32004811dd000482fb00cd
:102468000402410013017800820f52008d013200ee
:102478000200e000d5fe320064804100efe89700da
:102488008001780010017800820f52008401320028
:10249800640040000200e000f9ff3a001ac0b300ef
:1024a800d6fe370088189000287090006f406000b2
:1024b800e24f5000500132003a013e00e14f500017
:1024c8000e0032007fa897008fb097001fb19700c9
:1024d800afb1970040149800511498006214980006
:1024e800731498001c4678003c7c98001980fb0007
:1024f800201c98000045eb00b4fe3700114078001e
:102508000082fb008002eb006033b800f4af9f004c
:1025180085b79f0096b79f00a7b79f007fa8970031
:102528008fb097001fb19700afb197004014980083
:10253800511498006214980073149800e9ff37004a
:102548000ec545006ffe3700e4cf5500f400320099
:10255800e8cf5500a8fe3a008e81fb008381440035
:1025680083bf9f00134590000a80fb008000eb00aa
:102578006011b800c819dd004812de00830172003e
:102588004811dd00480ade0002017200c808dd00bb
:102598004802de00810072004800dd00b0b79f00ed
:1025a800c1b79f00d2b79f00e3b79f008fba9700cb
:1025b800254090000082fb008002eb006033b800e9
:1025c8008603780005037800840278000002eb0097
:1025d8003fb09700cfb097005fb19700efb1970079
:1025e80004004000858048000601490087814900b1
:1025f800b0af9f00c1af9f00d2af9f00e3af9f0075
:102608008fb89700114278000480fb008000eb002f
:102618006011b8003faa9700cfaa97005fab970058
:10262800efab97000002420081824a0002034b0090
:1026380083834b00b4b79f00c5b79f00d6b79f00f0
:10264800e7b79f008fba9700354290000480fb00df
:102658008000eb006011b800c811dd00480ade00f8
:10266800830172004809dd004802de0002017200a1
:10267800c800dd000000eb003fb29700cfb2970022
:102688005fb39700efb397000000420081804a00d3
:1026980002014b0083814b00b0af9f00c1af9f0088
:1026a800d2af9f00e3af9f008fba970045429000da
:1026b8000480fb008000eb006011b8000001be0040
:1026c8006000b8003faa9700cfaa97005fab9700b9
:1026d800efab97000000420081804a0002014b00e6
:1026e80083814b00b0b79f00c1b79f00d2b79f004e
:1026f800e3b79f008fba9700554290000480fb0013
:102708008000eb006011b800c809dd004802de0057
:10271800830172004801dd006000b8003fb29700f5
:10272800cfb297005fb39700efb397000000420065
:1027380081804a0002014b0083814b00b0af9f00ab
:10274800c1af9f00d2af9f00e3af9f008fba970041
:10275800654290000480fb008000eb006011b80027
:10276800800178000001eb006000b8003faa9700e4
:10277800cfaa97005fab9700efab9700000042002d
:1027880081804a0002014b0083814b00b0b79f0053
:10279800c1b79f00d2b79f00e3b79f008fba9700d9
:1027a800754290000480fb008000eb006011b800c7
:1027b800c801dd000001eb006000b8003fb29700df
:1027c800cfb297005fb39700efb3970000004200c5
:1027d80081804a0002014b0083814b00001498005d
:1027e800111498002214980033149800befd370085
:1027f8006bc0b30050002000410020008afd370064
:102808000b80fb0000804400204290003041900083
:10281800408f8000900178001ac0b3000300e000e8
:10282800eafd32004811dd000482fb000402410089
:1028380013017800820f5200900032000200e0007d
:10284800e2fd320064804100efe8970080017800e3
:1028580010017800820f52008700320064004000a7
:102868000200e000f9ff3a001ac0b300e3fd3700a8
:102878008b80fb008180440001017800b24378001e
:1028880012437800a1419000b1409000458f80002c
:1028980015017800004578000200e000cbfd320009
:1028a800c808dd008381fb00838140009200780026
:1028b800818f5100850032000100e000c3fd320025
:1028c800640041000001780090007800818f510079
:1028d8007e003200640040000100e000f9ff3a0089
:1028e8001ac0b300c5fd37008e81fb000382440087
:1028f8008401e8009381fb00c819dd001482fb0005
:10290800048241008002eb006033b8000414980090
:1029180015149800261498003714980072fd370093
:102928008e81fb00838144000302e8001482fb00cf
:102938008002eb00482bdd00c823de00870373000c
:102948004823dd000382e8001482fb008002eb00cc
:10295800c022dd00040020000603420087834a00ed
:102968001382fb008002eb000603420087834a00c3
:10297800e38141001382fb008002eb00c822dd00e6
:10298800040020000602420087824a006033b80033
:102998000414980015149800261498003714980009
:1029a80051fd3700e44f500023003200e84f50003b
:1029b800c4fe3a00110278009102900021039000b1
:1029c800b1039000f4af9f0085b79f0096b79f00b2
:1029d800a7b79f007fa897008fb097001fb19700f7
:1029e800afb19700401498005114980062149800f1
:1029f80073149800bbfe3700110078006102b8001c
:102a08006033b800f4af9f0085b79f0096b79f006a
:102a1800a7b79f007fa897008fb097001fb19700b6
:102a2800afb19700401498005114980062149800b0
:102a380073149800abfe37001102780091029000e1
:102a48006033b800f4af9f0085b79f0096b79f002a
:102a5800a7b79f007fa897008fb097001fb1970076
:102a6800afb1970040149800511498006214980070
:102a7800731498009bfe3700e1ef9f001ac0b30063
:102a88000200e00051fd3200130090000000e00059
:102a98004efd3200001c98006feb970001fd3700d7
:102aa800e1ef9f001ac0b3000200e00047fd3200ca
:102ab800130090000000e00044fd32001000780090
:102ac800001c98006feb9700f6fc37001ac0b300a3
:102ad8000100e0003dfd3200120290000400e00019
:102ae8003afd3200940178001501900092007800b8
:102af800818f51000c0032000100e00033fd3200ec
:102b08006c0041000001780090007800818f51002e
:102b1800050032006c0040000100e000f9ff3a00b7
:102b28001ac0b30035fd37001ac0b3000100e00039
:102b380026fd32000200e00024fd3200c830dd002e
:102b48000780fb008080400052019000040078005c
:102b580002000100001c98000000e0001bfd32008c
:102b6800a8729000e5ef9f0005437800cdfc370080
:102b7800e44f500023003200e84f500088fd3a002f
:102b8800110278009102900021039000b103900097
:102b9800f4a79f0085af9f0096af9f00a7af9f0047
:102ba8007fa097008fa897001fa99700afa997004b
:102bb80040149800511498006214980073149800f7
:102bc8007ffd3700110078006102b8006033b8005b
:102bd800f4a79f0085af9f0096af9f00a7af9f0007
:102be8007fa097008fa897001fa99700afa997000b
:102bf80040149800511498006214980073149800b7
:102c08006ffd370011027800910290006033b80020
:102c1800f4a79f0085af9f0096af9f00a7af9f00c6
:102c28007fa097008fa897001fa99700afa99700ca
:102c38004014980051149800621498007314980076
:082c48005ffd370000000500ec
:020000040000fa
:102c5000889fbe008a1f780000047800851b07004b
:102c6000c83092000100500050349a0008007800eb
:102c7000ba15070008007800d41307000800780090
:102c8000261a070008007800b4180700791b07000f
:102c9000c83092000100500060349a001830920051
:102ca000e30f50007c003a00a8349100e58f5400f7
:102cb0000d003200281892000000e00005003a00e4
:102cc0001100200008007800d21907000004e0007d
:102cd0000500320028189200310120000008a300ee
:102ce0000c003a000500370008e892008000eb0075
:102cf0000004e000150032000e0037004101200002
:102d00000018a30003003a000028a300ca02320002
:102d100021012000001720000800400018f992004f
:102d2000590020000204e00076003a007c1a0700f7
:102d30007400370058309100c500de004400de000a
:102d400080806800e18060000100a20008209200fd
:102d5000120020000008a30003003200482992005e
:102d60004311de00610161000000eb000104e0009e
:102d7000010032000280fb00e28f54001a00320092
:102d800005003e000900e00009003200e18f540018
:102d900033003a0011003700e48f54001b0032006a
:102da00017003900e58f54002d003a002800370045
:102db000002b20000800400010457800202b200048
:102dc00008004000890d07000a04e0004d003200b1
:102dd0000004e00024003a004a0037000004e0004c
:102de00023003a00470037000004e00022003200d0
:102df00018d892000004e00021003a00410037009a
:102e00000004e000200032003e00370018889200e5
:102e1000788192008889920000015100e081590078
:102e20006026200008004000904078000048eb0039
:102e3000e00f5100e08f5900870234000104e000e8
:102e400085023a0072849a00038c9a002d003700a4
:102e500008e892000004e0000d003a002900370065
:102e60008004eb00270037004900200025003700d0
:102e700029002000230037004900200021003700ee
:102e8000390020001f003700490020001d003700d6
:102e90008004eb001b003700281d92000af0a700f9
:102ea0000a05ea000a05ea004f55de000a04e000c0
:102eb00007003200001720000800400098f8920038
:102ec0000104e00002003a008000eb00141a070041
:102ed00018309200690020000000e0000900320074
:102ee0007026200008004000890020001004e00047
:102ef00004003a00790020000a04e00001003200da
:102f000069002000db1a0700c83092000100500061
:102f100070349a002830910080806c0001f0a70086
:102f20008100ea008100ea00cf08de002934990020
:102f3000e48f5400ee00320008003e00e18f5400a0
:102f4000780032000d003900e28f54008c0032000e
:102f5000e38f540007023a00c3003700e68f5400a5
:102f60005501320023013900e78f5400d0013200af
:102f7000e88f5400ff013a007c0137000104e000b3
:102f800052003200202b2000080040004b1a07009e
:102f9000c3fe2f0020618000008261001401b30095
:102fa000e2c1200010322400d1bc2a0045c220001a
:102fb0000109780000097800840a78002562800001
:102fc000058261001401b30045c4200001097800a6
:102fd00000097800840a78002463800084816100fd
:102fe0001301b30045c620000109780000097800ec
:102ff000830a7800002b2000080040000048eb0006
:10300000789092000000e00002003a0010002000da
:1030100070949a008044eb0009ec9a0000c1b30060
:1030200000fc9a0019fc9a0040242000080040008f
:10303000e718070000d0270050049900f000200096
:10304000600499002000200070049900683091000d
:103050006011b8003214990043149900781091005f
:10306000cf80de00c000dd00000020005014990079
:10307000611499000000eb00302c9900622c99003b
:10308000732c990010dc9a0009dc9a0029dc9a0064
:1030900040002000600c9900e0172000080040006c
:1030a0006d180700e0222000080040000948780061
:1030b0000023200008004000c319070060232000ff
:1030c00008004000d0190700aa013700789092004c
:1030d0000000e0000c0032000000e90070949a004b
:1030e000a4013a00218ca900218ca8001000200026
:1030f000e016070020002000de1607003000200048
:10310000dc1607009b0137006c01440041292000b8
:1031100088804000002a200008004000f8150700c1
:10312000940137000104e0000e003200080078002e
:10313000221a0700781892000010a000701c9a0054
:10314000e01720000800400043180700e02220009c
:10315000080040000048eb00002320000800400069
:10316000321a070008e892000004e00081013a00ea
:1031700060232000080040009b1907007d013700f4
:103180000104e0002600320008007800561707000e
:103190006000b800500c9800610c98006014980012
:1031a0007114980020bc980031bc9800e0222000e7
:1031b0000800400011c0b300014878005000200012
:1031c00030618800306288003063880013618000bd
:1031d0000390a100e2c1200010322400d1bc2a00db
:1031e00024c220000109780000097800030a780051
:1031f000136280000390a10025c42000010978001b
:1032000000097800830a7800136380000390a1000e
:1032100024c620000109780000097800030a78001c
:1032200008007800bb0f070038319000e50f51000f
:103230000100310052002000c8309000e58f50009e
:10324000010031005100200058309000e50f50007f
:103250000100310050002000326188003162880096
:1032600030638800430137000104e0000e003200a3
:10327000e830910018019000cf91de00c011dd0010
:103280000200200022bc980033bc98006011b800f6
:10329000622c9900732c9900103b21008088b900a2
:1032a0004004990010bc980008007800990f0700ae
:1032b00038319000e50f510001003100520020002c
:1032c000c8309000e58f500001003100510020000f
:1032d00058309000e50f50000100310050002000f0
:1032e0003261880031628800306388002101370034
:1032f0000104e000380032000000eb0010bc980030
:10330000f3f32f001561800005826100e2c1200007
:1033100010322400d1bc2a0025c220000109780007
:1033200000097800840a7800156280000582610037
:1033300025c420000109780000097800840a78007b
:10334000146380008481610025c620000109780093
:1033500000097800830a7800136180000390a000c0
:1033600024c220000109780000097800030a7800cf
:10337000136280000390a00025c42000010978009a
:1033800000097800830a7800136380000390a0008e
:1033900024c620000109780000097800030a78009b
:1033a0008029200030618800306288003063880006
:1033b00058389200a00090008100e8002100980099
:1033c00058809200e880920070849a00018c9a00e4
:1033d00010002000108c9a0008e892000004e00021
:1033e000e4003a006023200008004000fe180700b7
:1033f000e00037000104e000de0032000040eb0096
:1034000000ec9a00f3f32f0011618000018261004b
:10341000e2c1200010322400d1bc2a0025c22000c5
:103420000109780000097800840a7800156280009c
:103430000582610025c42000010978000009780098
:10344000840a7800146380008481610025c620000e
:103450000109780000097800830a78001361800070
:103460000390a00024c22000010978000009780020
:10347000030a7800136280000390a00025c4200096
:103480000109780000097800830a7800136380003e
:103490000390a00024c620000109780000097800ec
:1034a000030a78008029200030618800306288009b
:1034b00030638800af003700f3f32f001561800000
:1034c00005826100e2c1200010322400d1bc2a0034
:1034d00025c220000109780000097800840a7800dc
:1034e000156280000582610025c420000109780072
:1034f00000097800840a78001463800084816100e8
:1035000025c620000109780000097800830a7800a8
:10351000136180000390a00024c2200001097800fc
:1035200000097800030a7800136280000390a0006d
:1035300025c420000109780000097800830a78007a
:10354000136380000390a00024c6200001097800c6
:1035500000097800030a7800802920003061880083
:103560003062880030638800820037000104e00088
:103570002c003200202b200008004000cf1807004c
:10358000c3fe2f0025618000058261001401b30095
:10359000e2c1200010322400d1bc2a0045c2200024
:1035a0000109780000097800840a7800256280000b
:1035b000058261001401b30045c4200001097800b0
:1035c00000097800840a7800246380008481610007
:1035d0001301b30045c620000109780000097800f6
:1035e000830a7800002b2000080040000048eb0010
:1035f000789092000000e00002003a0010002000e5
:1036000070949a006000b800500c9800610c98000b
:10361000601498007114980020bc980031bc980088
:1036200054003700789092000000e0001c00320047
:103630000000e90070949a004e003a00218ca90025
:10364000218ca800c3ff2f00206180000082610050
:10365000e2c1200010322400d1bc2a0045c2200063
:103660000109780000097800840a7800256280004a
:103670000582610045c42000010978000009780036
:10368000840a7800246380008481610045c620009c
:103690000109780000097800830a780035003700b6
:1036a00070262000080040000048eb003100370081
:1036b0000104e0001e003200c82892000158a30057
:1036c00002003200e20f50001900320050002000ca
:1036d00030618800306288003063880013618000a8
:1036e0000390a100e2c1200010322400d1bc2a00c6
:1036f00024c220000109780000097800030a78003c
:10370000136280000390a10025c420000109780005
:1037100000097800830a7800136380000390a100f9
:1037200024c620000109780000097800030a780007
:1037300008007800770e070038319000e50f51003f
:103740000100310052002000c8309000e58f500089
:10375000010031005100200058309000e50f50006a
:103760000100310050002000326188003162880081
:1037700030638800bf180700c83092000100500075
:10378000003c9a0008007800411607005838920063
:10379000c0009000601a2d00808f5000050032009c
:1037a0000000eb00402c9a003100200011349a00f8
:1037b000102c9a00182892000000e0001700320038
:1037c0004f80de00000040000000e8002829920041
:1037d000b829920061014100e0814900222c9a0041
:1037e000332c9a00282a9200b82a920028219200ad
:1037f000b8219200820f5200838f5a0006003900d0
:103800000000ea00102c9a006000b800202c9a00fa
:10381000312c9a0001003700102c9a0095180700ef
:10382000c830920001005000103c9a004f0578000b
:103830004f04be00000006001100200008007800c0
:10384000f4160700010120000004e00031fd3a00f9
:103850008000eb002ffd37006011b80072849a00e1
:0c386000038c9a0019002000a6fd370020
:020000040000fa
:10386c0021c0b30041409800b000900012c2b300d8
:10387c00924098009000900001040100504190008b
:10388c00d1c2b300814f5100bb003600e2c2b3007d
:10389c0042409800b00190000041eb00924198002a
:1038ac00b001900054c0b300a4419800b001900046
:1038bc00b2419800428f8000a20990003001900024
:1038cc0043419800428f8000a20990003001900083
:1038dc00c819de005341980030019000d04190008f
:1038ec00634198003001900003c1b300734198000c
:1038fc003001900023c8b3000349980030019000b8
:10390c0043c4b300134998003001900053c6b30070
:10391c00234998003001900083c1e9003349980095
:10392c00b001900012c3b300c2499800b0019000de
:10393c0084c3b300d4499800b00190006642520091
:10394c00e44998003002900003c3b300734a980016
:10395c0030029000025298003002900095c3b300e0
:10396c0015529800300290002252980030019000bd
:10397c003351980030019000e3c14100435198004d
:10398c00300190008341e80053519800428f800031
:10399c00b20990000300e0007e0032003209900072
:1039ac00b000900012417800e2509800418f8000e6
:1039bc0031099000b000900012419000f250980034
:1039cc00418f800031099000b0009000224190009e
:1039dc0082589800418f800031099000b00090000f
:1039ec004241900092589800418f8000310990001c
:1039fc00b000900052419000a2589800418f800076
:103a0c0031099000b000900072419000b2589800bb
:103a1c00418f800031099000b00090000249900065
:103a2c00c2589800418f800031099000b00090007e
:103a3c0012499000d2589800418f800031099000b3
:103a4c00b000900022499000e2589800418f80000d
:103a5c0031099000b000900032499000f258980063
:103a6c00418f800031099000b000900042499000d5
:103a7c0082609800418f800031099000b000900066
:103a8c006249900092609800418f8000310990004b
:103a9c00b000900072499000a2609800418f8000a5
:103aac0031019000b0009000b2609800418f80000e
:103abc0041019000b0009000c2609800418f8000de
:103acc0041019000b00090004811de00d2609800d7
:103adc00418f800051019000e1019000b0009000f6
:103aec00e2609800418f800051019000e10190004c
:103afc00b0009000481add004811de00020172008f
:103b0c00c819de00f2609800418f800051019000ce
:103b1c00e1019000b000900083689800418f800014
:103b2c0051019000e1019000b00090004819de00b6
:103b3c0092689800428f8000cf91de00b000900018
:103b4c00a2689800b0009000c81ade00481bdd0087
:103b5c004812de0004027300b4689800b0009000b4
:103b6c00c3689800b00090004819de00d268980035
:103b7c00900090000104010021c0b3004140980066
:103b8c00b000900052c1b300924098009000900099
:103b9c000104010030019000216198003001900077
:103bac001161980030019000016198003001900083
:103bbc0071599800300190006159980030019000c3
:103bcc0051599800300190004159980030019000f3
:103bdc003159980030019000215998003001900023
:103bec001159980030019000015998003001900053
:103bfc00715198003001900061519800418f800004
:103c0c0031019000b0009000b2609800418f8000ac
:103c1c0041019000b0009000c2609800418f80007c
:103c2c0041019000b00090004811de00d260980075
:103c3c00418f800051019000e1019000b000900094
:103c4c00e2609800418f800051019000e1019000ea
:103c5c00b0009000481add004811de00020172002d
:103c6c00c819de00f2609800418f8000510190006d
:103c7c00e1019000b000900083689800418f8000b3
:103c8c0051019000e1019000b00090004819de0055
:103c9c0092689800428f8000cf91de00b0009000b7
:103cac00a2689800b0009000c81ade00481bdd0026
:103cbc004812de0004027300b4689800b000900053
:103ccc00c3689800b00090004819de00d2689800d4
:103cdc009000900001040100881f78000004780017
:103cec00b800900021429000810378005740780082
:103cfc00428f8000920278000500e00088003200bc
:103d0c004822dd000080fb00000242009501780093
:103d1c00830f5200130032000300e0000800320051
:103d2c00648042008002780090017800830f52007a
:103d3c000c003200640040000300e000f9ff3a0080
:103d4c0000c4b30021c0b30041449800804b7800fc
:103d5c009800900008007800010001004f047800e2
:103d6c00000006000300e000f5ff32001500900093
:103d7c00a20190000300e0001a003200a2029000a1
:103d8c008001eb00950f120012003200a20290008d
:103d9c00430020001500e00074003200a2029000e5
:103dac0083824200950f12000a003200a20290009a
:103dbc0064834100838242001500e000050032005c
:103dcc0086017800a202900083824200950f1200b7
:103ddc00f6ff3a0022029000030242001400e000b9
:103dec003b003a00920190000300e00065003200b5
:103dfc0010037800120290008001eb00940f130066
:103e0c0012003200120290001400e0000f00320089
:103e1c00c30020001202900003024200940f130012
:103e2c000a00320012029000ec82410003024200b0
:103e3c001400e000050032008501780012029000a9
:103e4c0003024200940f1300f6ff3a001202900096
:103e5c00030242001400e000130032001201900033
:103e6c00830141004841900063415100e3804000d0
:103e7c00c3019000030001000004e00030003a0090
:103e8c0021c0b30041449800b800900090409800c5
:103e9c009800900008007800010001004f047800a1
:103eac0000000600afff370020c0b300404498006c
:103ebc0010c4b300804b7800980090000800780084
:103ecc00010001004f04780000000600a5ff370038
:103edc002201900083014100484190006341510050
:103eec00e380400093019000030001000004e00017
:103efc009aff320020c0b300404498003800900074
:103f0c0021c4b3001140980098009000080078007c
:103f1c00010001004f0478000000060091ff3700fb
:103f2c0030c4b30021c0b30041449800804b7800ea
:103f3c0098009000080078000100010087ff37000e
:103f4c0020c0b300404498003800900041c1b30039
:103f5c0011409800980090000800780001000100c2
:103f6c004f047800000006007eff37008001eb0054
:103f7c0022029000030242001400e00099ff32007c
:103f8c00d3ff370020c0b3004044980040c4b300b6
:103f9c00804b780098009000080078000100010028
:103fac004f047800000006006eff3700881f780071
:103fbc0000047800380390008680e8009142780075
:103fcc0056407800438f8000130278000400e00014
:103fdc0053003200c82add000080fb0080824200c2
:103fec0014017800828f5200130032000200e000ae
:103ffc0008003200640042000002780010017800d2
:10400c00828f52000c003200640040000200e0007d
:10401c00f9ff3a0000c4b30021c0b300414498003a
:10402c00004b780098009000080078000100010017
:10403c004f047800000006000200e000f5ff32009b
:10404c0014009000130190000200e0003c003200cc
:10405c0090037800130290000001eb00948f130082
:10406c0012003200130290001400e0000f00320026
:10407c00c20020001302900002024200948f130031
:10408c000a00320013029000ec02410002024200ce
:10409c001400e000050032000501780013029000c6
:1040ac0002024200948f1300f6ff3a0013029000b4
:1040bc00020242001400e0000f0032009301900055
:1040cc0002814100320190000200010000c0e800b2
:1040dc0040449800380090008040eb00114098005c
:1040ec009800900008007800010001004f0478004f
:1040fc0000000600d0ff370020c0b30040449800f9
:10410c0010c4b300004b78009800900008007800b1
:10411c00010001004f04780000000600c6ff3700c4
:10412c0030c4b30021c0b30041449800004b780068
:10413c00980090000800780001000100bcff3700d7
:10414c0020c0b3004044980040c4b300004b78003a
:10415c009800900008007800010001004f047800de
:10416c0000000600b4ff3700b00090005141780009
:10417c00e24f5100380032000c003600e44f510081
:10418c003f0032001e00310033002000428f8000bf
:10419c00330198000041eb008248780021c0b30045
:1041ac004140980090009000010401000204e000de
:1041bc000a003a008001eb00428f80003301980026
:1041cc000041eb008248780021c0b30041409800c8
:1041dc009000900001040100f4ff3700e14f510002
:1041ec001300320022c2b3008248780021c0b30011
:1041fc00414098009000900001040100ebff370053
:10420c00e54f5100f7ff3a0053002000428f800029
:10421c00330198000041eb008248780021c0b300c4
:10422c00414098009000900001040100dfff37002e
:10423c0013002000428f8000330198000041eb00f6
:10424c008248780021c0b300414098009000900053
:10425c0001040100d5ff370023002000428f8000ad
:10426c00330198000041eb008248780021c0b30074
:10427c00414098009000900001040100cbff3700f2
:10428c0043002000428f8000330198000041eb0076
:10429c008248780021c0b300414098009000900003
:1042ac0001040100c1ff3700b00090000041eb0099
:1042bc0092409800418f800031019000b000900036
:1042cc00a240980031c0b30041409800900090008b
:1042dc000104010022c0b30042409800300190005c
:1042ec001141980090009000010401002117210059
:1042fc00630320008181410062c321008228780081
:10430c00838f5000fdff3a004117210041009800b7
:10431c00000006004000900041c421000108780014
:10432c00a115220011009800a10b22002100980079
:10433c0021e7210021109800c1fd210011109800e7
:10434c000000060011002000110898008000eb000e
:10435c000108980000000600e4874700889fbe0013
:10436c008a9fbe008c9fbe008e1f780000047800d0
:10437c00980c90005ac5b3003b002000e18f54000c
:10438c0015003a0058009000b000900001000100a8
:10439c000004e0002300320008089000e20f5000f7
:1043ac000801320058003e000000e000a0003a0076
:1043bc004a5498005054980058009000100178000e
:1043cc008a40780002000100090c9800980c9000bb
:1043dc00e18f5400ebff32000900e00014003a00ba
:1043ec0058009000a0009000010001000004e000c3
:1043fc000f00320058009000900090000100010066
:10440c00f8009000e28f5000b800320017003e0018
:10441c000100e00064003a0051c5b300814f500028
:10442c001c013200980c90000900e000ecff3200f7
:10443c006a064400408f8000c00890000100e00034
:10444c0004003200c0089000a1189000e48f5000c6
:10445c004e0132004f0778004f06be004f05be00dc
:10446c004f04be004f00b10000000600e48f500066
:10447c008100320086003900e58f500004003200c4
:10448c000000eb0070049800980c9000e6ff3700d9
:10449c00c850900052c5b30082cf500011003200ba
:1044ac00e2cf50000f003200814f500011003a0053
:1044bc003800900010407800fa4f5000fa003e008f
:1044cc000080fb00c800900000004000008040000d
:1044dc00900078000800780001000100980c900012
:1044ec00d1ff370081c0ea0041549800814f500041
:1044fc00efff320031c1b3000800780075ff0700f0
:10450c00980c9000c8ff3700e40f50008600320072
:10451c008d003900e50f5000050032000000eb0063
:10452c00100c9800700498008004eb00acff37006e
:10453c00c850900050c5b30080cf50000d00320021
:10454c00e2cf50000b0032005800900010017800b0
:10455c000200010058009000d00090000100010002
:10456c000000eb00100c9800700498008004eb0025
:10457c009bff370081c0ea0041549800580090001e
:10458c00100178000200010058009000d00090004b
:10459c00010001000000eb00100c98007004980062
:1045ac008004eb008eff3700e18f5000b4ff3a001f
:1045bc000004e0001b003200d8409000814f5000f6
:1045cc00de003e0052c5b3008240400041549800ca
:1045dc004044980059549800210020007104980020
:1045ec0082407800814f500002003200e24f5000b0
:1045fc008cff3a00d4f1b70020002000508f8800c7
:10460c004000200070049800980c900086ff370042
:10461c0051c5b300421d210012417800814f510059
:10462c00ce00320079049800980c90007eff370081
:10463c00e10f5000b9ff3a00c8409000485090007c
:10464c000140400040549800580090001001780040
:10465c0002000100484090008a4f50008600320052
:10466c00e24f50008400320020002000000c980023
:10467c00980c900041ff37000004e000e4ff3a0082
:10468c00508f800070049800980c900066ff3700e3
:10469c00c850900080c0400041549800d850900001
:1046ac008180fb0038019000810041008048780037
:1046bc00d85090008140e800515498004841900037
:1046cc0082cf50004e00390051c5b300814f5000cd
:1046dc007a003200e24f5000780032005000200087
:1046ec0070049800980c90004fff3700c848900059
:1046fc0080cf5000cbff3a00485090000140400062
:10470c004054980050c5b30080cf50008300320055
:10471c00e2cf50008100320030002000700498007d
:10472c00980c900040ff3700580090001001780062
:10473c008040eb0002000100508f8000000c9800bc
:10474c00980c90000dff3700d85090008180fb0032
:10475c00380090008100400048509000114040000b
:10476c004054980058009000100178009140780057
:10477c0002000100d85090000180fb008001e8008d
:10478c00484190000281fb00828f510028003500c7
:10479c003801900000004100104078008a4f500012
:1047ac0055003200e24f5000530032005000200000
:1047bc00000c98008140e80051549800980c90002f
:1047cc00eefe3700c8489000485090000140400071
:1047dc00405498005800900010017800020001002d
:1047ec00484890008a4f50001d003200e24f5000a4
:1047fc001b0032000b0c9800980c9000dffe370069
:10480c0051c5b300814f500002003200e24f5000fe
:10481c00c1ff3a00d4f1b70030002000508f88005f
:10482c004000200070049800980c9000fefe3700a9
:10483c003801900000004100104078008a4f500071
:10484c0025003200e24f5000230032000b0c980080
:10485c008140e80051549800980c9000c7fe370036
:10486c00d4f1b7005b8f880040002000000c98004a
:10487c00980c9000c1fe3700d4f1b7002000200046
:10488c00508f880040002000000c9800980c90007d
:10489c00bafe3700405498001000200070049800b5
:1048ac00980c9000e0fe370011c2b30008007800ad
:1048bc0088fe0700980c9000dbfe3700d4f1b7009f
:1048cc0050002000508f8800400020007004980099
:1048dc00980c9000d4fe3700d4f1b7005b8f8800a1
:1048ec0040002000000c98008140e80051549800d2
:1048fc00980c9000a1fe3700d4f1b70050002000b6
:10490c00508f880040002000000c98008140e80087
:10491c0051549800980c900098fe3700401d2100cf
:10492c000148780030002000508f880040002000a3
:10493c0070049800980c9000bbfe37007904980026
:10494c00380090000048eb0051c1b300080078001b
:10495c0060fe0700980c9000b3fe3700d840900022
:10496c00814f5000f5ff3e0052c5b300824040001d
:10497c00415498004044980059549800200020005d
:10498c0070049800980c9000a7fe37004008900027
:10499c00a0c490008984fb00e3844400580090007c
:1049ac00c0009000010001000080fb00808f5400cb
:1049bc0007003d00408f800040099000c008900027
:1049cc0072199000e1189000810f51000d00310018
:1049dc00b08e8000c18e800061004000e0804800f5
:1049ec00b08e8800c18e88004f0778004f06be003d
:1049fc004f05be004f04be004f00b1000000060082
:104a0c009afe3700400890008000eb007118980067
:104a1c00580090001001780021c0b3000200010082
:104a2c0058009000418f8000c1089000a1c09000f8
:104a3c00100178000200010058009000c848900056
:104a4c00100178000200010058009000418f800096
:104a5c00c108900081209000100178000200010034
:104a6c0058009000418f8000c10890008120900078
:104a7c00c808de001001780002000100408f8000a1
:104a8c00c0099000c00890004009900023c290001b
:104a9c00c84990008341420083c1e8008120900006
:104aac0081c0410092c5900081c545000007eb0014
:104abc008004eb008e00e80081bf9f007207470066
:104acc0081864000400890000d004000108044009a
:104adc00104578001c007800100178008a4078009e
:104aec00020001008ac545008904e800408f80005f
:104afc00c00890008e8040009180fb00818f540094
:104b0c00f0ff39000fbf9700c0089000b1789000fb
:104b1c008180fb00810f5700e5ff3900e2cf550083
:104b2c000b00320058009000100178008b40780088
:104b3c00020001004f0778004f06be004f05be0073
:104b4c004f04be004f00b1000000060047fe3700c6
:104b5c00dbcfb30058009000100178008b40780038
:104b6c0002000100f3ff370031009800524098001a
:104b7c0043489800211b220001087800811a22006a
:104b8c00110098008000eb0011089800710098004b
:044b9c00000006000f
:020000040000fa
:104ba000889fbe008a9fbe008c9fbe008e1f78002b
:104bb00000077800310a900004a2b9000402420004
:104bc00085824a000501780002f0a7000281ea0010
:104bd000410b900006b3b9000603430087834b00e6
:104be0000702780004f0a7000482ea0002014200f4
:104bf000122f98005e239000ee239000ce219000ab
:104c00000392b9000402430085824b007e2390008a
:104c100003b3b9000602520087825a005427980055
:104c2000652798004128dd004f21de000201700059
:104c300002037800722798000e2a900004a2b9009f
:104c40000402420085824a000501780002f0a700b4
:104c50000281ea00820f5300120034002e299000d6
:104c6000be29900061014100e0814900222f980097
:104c7000332f98004e2a9000de2a9000840f5100b6
:104c8000858f59000a0039006011b800222f980062
:104c9000332f98004e9190000200a0004297980098
:104ca000060037006011b800222f9800332f9800bb
:104cb0004e9190000200a100429798003129910086
:104cc000e10f51009f013200e30f51009d013200be
:104cd000e40f51009b01320061399200e20f510054
:104ce0001b003a006e2990009e0f110018003d0035
:104cf0001200200003002000722f98000337980054
:104d00003e319000ce31900061014100e0814900c8
:104d100032379800433798005e329000ee329000b0
:104d2000840f5100858f5900220036006011b800b1
:104d30003237980043379800722f98000337980055
:104d40004e9190000230a000429798001c0037005e
:104d50003e319000ce319000e00f5100e08f5900bd
:104d60001400320061014100e081490032379800af
:104d7000433798007e2990008e31900061014100f8
:104d8000e0814900722f9800033798001e3290008e
:104d9000ae329000840f5100858f59000500360017
:104da0006011b8003237980043379800722f98008e
:104db000033798004e9190000230a100429798006e
:104dc0009e0278001e1b9000ae1b9000fe1190000a
:104dd00003bcb9000803530089835b0003adb9002d
:104de0000601450087814d00121f9800231f98007f
:104df00003037800850178004fb1de0002f0a200c5
:104e0000868151004240af0082017800031f980064
:104e10001e0290005e1b9000ee1b90003e19900059
:104e200002bcb9000804530089845b0002a6b900e3
:104e30000804460089844e00581f9800691f980096
:104e4000040178004fccde0008f0a20009015100f7
:104e50004240af0008017800421f9800039cb9004f
:104e60000804440089844c008901780003f0a700fd
:104e70008381ea000294b9000804440089844c004c
:104e80000901780002f0a7000281ea000e149000e8
:104e90009e14900003014100fe0b90000791b900a1
:104ea0000201440083814c002e14900007c4b90015
:104eb00008035100898359000617980017179800b6
:104ec000413cdd004f31de000201740022179800e2
:104ed00005abb9000603430087834b000701780048
:104ee00002f0a7000281ea0004a2b9000402420015
:104ef00085824a008501780003f0a7008381ea00db
:104f00000e0b90009e0b900002814100fe0290006b
:104f10000591b9000201430083814b002e0b9000e4
:104f200005b3b9000602510087825900040f9800aa
:104f3000150f98004128dd004f21de0002017000ae
:104f4000220f980021319100e30f5100b7003a0081
:104f5000f130900001f0a7008100ea0001f0a70005
:104f60008180ea007e319000828f500018003d0061
:104f70001200200003002000023f9800133f980019
:104f80004e399000de39900061014100e081490016
:104f9000423f9800533f98006e3a9000fe3a9000ce
:104fa000840f5100858f5900220036006011b8002f
:104fb000423f9800533f9800023f9800133f9800eb
:104fc000ce9090000120a000419798001c0037006f
:104fd0004e399000de399000e00f5100e08f59000b
:104fe0001400320061014100e0814900423f980015
:104ff000533f98000e3990009e39900061014100a6
:10500000e0814900023f9800133f98002e3a90003b
:10501000be3a9000840f5100858f5900050036007c
:105020006011b800423f9800533f9800023f98003b
:10503000133f9800ce9090000120a1004197980066
:10504000ee00900001f0a7008180ea002e89900018
:10505000828f500057003d002e02900004a2b9003c
:105060000402420085824a000501780002f0a70090
:105070000281ea003e03900006b3b9000603430034
:1050800087834b008701780003f0a7008381ea0043
:10509000028541000a8798004e0190000291b900f4
:1050a000020141008381490003f0a7008381ea00e7
:1050b0005e03900006b3b9000603430087834b00ec
:1050c0000702780004f0a7000482ea00030442000b
:1050d000188798002e9190000191b90002014100bb
:1050e000838149001e9290000302420001a2b90090
:1050f0000402420085824a000e929000050142009f
:10510000528f98000a92b9000402420085824a0038
:1051100005017800658f98003e8b900001b3b900bf
:105120000603430087834b00478f980008bab900f5
:105130000403420085834a00778f9800828f5300d2
:105140001c003400110009000710d900000178008c
:105150003297980012002000030020002287980058
:10516000338798006e819000fe81900061014100bc
:10517000e081490062879800738798000e8a90004a
:105180009e8a9000840f5100858f590024003600bc
:105190006011b80062879800738798002287980092
:1051a00033879800ce9090000140a000419798006e
:1051b0001e003700f1ff2700319798006e819000a4
:1051c000fe819000e00f5100e08f59001400320082
:1051d00061014100e081490062879800738798006f
:1051e0002e819000be81900061014100e081490064
:1051f00022879800338798004e829000de829000cc
:10520000840f5100858f5900050036006011b800e9
:1052100062879800738798002287980033879800e8
:10522000ce9090000140a10041979800ee90900030
:105230008100e800619798007e919000828f500075
:10524000400039008000eb00619798004e119000fb
:10525000de1190002e129000be10900001a2b90045
:1052600004024100858249006e1190000191b9004d
:105270000202520083825a00441798005517980082
:10528000412bdd004f21de00020173006217980000
:105290004e0a9000de0a90002e0b9000be0890008f
:1052a00001b3b9000603420087834a006e0a9000ea
:1052b00001a2b9000403530085835b00460f9800e8
:1052c000570f9800413cdd004f32de0004027400ad
:1052d000640f980044a2de00741f9800820f5200f1
:1052e00012003d000e2190009e21900061014100be
:1052f000e081490002279800132798002e22900091
:10530000be229000840f5100858f59000a00390099
:105310006000b8000027980011279800ce909000f8
:105320000110a00041979800060037006011b800f6
:105330000227980013279800ce9090000110a1003a
:10534000419798004f0778004f06be004f05be00fa
:085350004f04be00000006003e
:020000040000fa
:10535800889fbe005011900002f0a7000201ea00e9
:1053680002f0a7000281ea0043552500830f51008f
:105378003a003c0060099000670151006701610034
:10538800ed014100c219dd008301400021029000b7
:10539800130252004211dd006203b0000201400016
:1053a800b101900092815100700190008202ea00e0
:1053b800820f520005003c0005037800848f5200dc
:1053c80003003d0004037800010037000203780061
:1053d800828f510004003c0005017800830f5100c2
:1053e80001003d0003017800b0019000069bb90060
:1053f800c139dd004f32de0004827100cfbade0011
:1054080084017800050478004f9ade00850f520069
:105418000300320008027800f5ff270085016a00c2
:1054280023309800b00190000299b900411bdd00bb
:105438004f12de0004027300cf9ade0004047800e5
:105448004fc2de00850f520002003200f2ff270033
:1054580002846a00383098003900370060099000eb
:10546800ed014100c219dd008301400021029000d6
:10547800130252004211dd006203b0000201400035
:10548800b101900092815100000990008202ea0067
:10549800820f520005003c0005037800848f5200fb
:1054a80003003d0004037800010037000203780080
:1054b800828f510004003c0005017800830f5100e1
:1054c80001003d0003017800b0019000069bb9007f
:1054d800c439dd004c32de0004827100ccbade0033
:1054e800840178004f9ade00850f520004003200d4
:1054f800cfbade0005027800f5ff270085016a00b3
:1055080023309800b00190000299b900441bdd00d7
:105518004c12de0004027300cc9ade00040478000a
:105528004fc2de00850f520004003200cf9cde001f
:1055380009047800f2ff270002046c003830980054
:10554800600990000201e8006701610062089800a4
:10555800ed014100c219dd008301400021029000e5
:10556800840978004211dd000201400031039000f7
:105578003619980020019000210390000693b90085
:10558800413add004f31de0002017200cfb9de0082
:10559800020278004fa1de00830f510002003200a2
:1055a800f2ff270002826900443098000019900039
:1055b800cf91de00cfa2de0004025100858259009f
:1055c80020319000cf91de000202520083825a00ff
:1055d8008582d1000482d3003428980020019000ed
:1055e800310390000693b900413add004f31de00e7
:1055f80002017200cfb9de00020278004fa1de007e
:10560800830f510002003200f2ff27000282690076
:105618005430980010199000cf91de00cfa2de0020
:10562800040251008582590030319000cf91de008c
:105638000202520083825a008582d1000482d3007c
:1056480044289800110378000618980091009000eb
:105658001118980010019000d00890000101410035
:1056680012309800010820000209b8008300780071
:105678000200e00010003a0001814000038022008f
:105688000281410012017800023098000102b00046
:10569800f2072000828f5000010036000108b10097
:1056a8008180400002802200810041009100780042
:1056b800712898002500370081814000048022006d
:1056c80083014200930178008100e800f40720007c
:1056d800848f5000010036000108b10001824000ab
:1056e8000580220004824200148211000492b8004e
:1056f8008581410003309800ff804000f3072000b7
:10570800838f5000010036000108b10081814000fc
:105718000480220083014200930178008100e800a0
:10572800f4072000848f5000010036000108b10002
:105738008180400004802200810042001182110013
:105748000492b8008581410073289800b028900021
:10575800702b9000068ab900c02990000031900093
:10576800029cb9000804420089844a0008044400e5
:1057780089844c0059289800069bb9000289b90011
:105788000201530083815b000203410083834900c7
:10579800070178006728980010139000a013900064
:1057a800f0089000018254009008900001a2b9000e
:1057b8000402430085824b001410980025109800bd
:1057c8000402420085824a00750898003013900050
:1057d800c013900000129000040151000191b9001b
:1057e8000201430083814b00321098004310980057
:1057f80002024100838249000502780005109800e2
:10580800501190008200780001f0a7008100ea00a2
:1058180001f0a7008180ea0093882000838f500060
:105828000500340011c0b3000500e00006003c008c
:105838008040eb000400370011c0b3000200e00014
:1058480001003c008040eb000104e000030032004e
:10585800f00890000102520002003700f0089000a2
:1058680001024200d0009000048ab900c528dd007a
:105878004b21de0002817000cba9de008200780097
:105888004f89de00830f510004003200cfa9de00eb
:1058980003017800f3ff270083006900212898009e
:1058a80030099000c0099000108ab9000402410034
:1058b800858249003408980045089800040242008f
:1058c80085824a005508980060119000f0119000f8
:1058d8005012900084805000200a9000048ab90079
:1058e80004024100858249006410980075109800f0
:1058f8000402420085824a00551098004f04be00f9
:045908000000060095
:020000040000fa
:10590c00881f780000047800380190008280e8003d
:10591c001180fb004800dd00124190000281fb0069
:10592c000200400010037800438f800013029000a7
:10593c000001eb00940f13001200320013029000d0
:10594c001400e0000f003200c2002000130290008f
:10595c0002024200940f13000a003200130290005e
:10596c00ec024100020242001400e000050032008b
:10597c00050178001302900002024200940f1300fc
:10598c00f6ff3a0013029000020242001400e000fd
:10599c000e00320093019000028141003201900010
:1059ac000200010000c0e80040449800380090005c
:1059bc008040eb001140980098009000080078009f
:1059cc00010001004f0478000000060011c4b30070
:1059dc00080078003ffa07004f047800000006002a
:1059ec00faff3700881f780000047800b800900098
:1059fc00214190004811dd00114090000080fb0017
:105a0c000000410010037800438f800013029000c7
:105a1c000001eb00940f13001200320013029000ef
:105a2c001400e0000f003200c200200013029000ae
:105a3c0002024200940f13000a003200130290007d
:105a4c00ec024100020242001400e00005003200aa
:105a5c00050178001302900002024200940f13001b
:105a6c00f6ff3a0013029000020242001400e0001c
:105a7c00180032009301900082814100484190004f
:105a8c0063415100e3804000c3019000030001001a
:105a9c000004e00009003a0021c0b3004144980022
:105aac00b800900090409800980090000800780092
:105abc00010001004f0478000000060041c1b30052
:105acc000800780003fa07004f0478000000060075
:105adc00faff370011c4b30008007800fdf9070085
:105aec004f04780000000600f4ff3700881f780090
:105afc003001900002047800b242900042439000c2
:105b0c000582fb008483e800d04190008381fb0078
:105b1c0051c1b300838f53000c003e00a241900092
:105b2c00c819dd00924090008180fb00818141000a
:105b3c00e24f530008003200e44f530033003200b0
:105b4c0041c1b300e14f530025003200e1f90700d9
:105b5c004f047800000006000400e000170032003b
:105b6c008000eb008180e8000101410013497800be
:105b7c003001900001014100330378004833de000e
:105b8c0016419800810f52000b0036003001900036
:105b9c008180e80001014100134978003001900038
:105bac0001014100330378004833de0016419800b0
:105bbc00810f5200f5ff3e003004900085c2e800d2
:105bcc00454098008040eb001144980090009000f4
:105bdc00010001004f04780000000600deff3700d2
:105bec000400e000f5ff32008000eb0001014100f1
:105bfc0033437800264198008100e800810f520061
:105c0c00edff360030019000f8ff37000400e00093
:105c1c00eaff32008000eb000101410013447800e0
:105c2c0028419800300190000101410013037800d5
:105c3c0093039000483cdd004833de0006037400fb
:105c4c00c83bde0036419800e480400030019000f3
:105c5c000101410023439000064978003001900077
:105c6c00010141003344900018419800e481410047
:105c7c00810f5200d0ff360030019000e6ff370054
:105c8c00889fbe008a1f780000057800ba04900037
:105c9c00890278009943900029429000ca419000f3
:105cac00e4c15100394190008381fb000283fb0069
:105cbc00110009008681d800010378000600e0007d
:105ccc0009003a004822dd008783fb0007024200ee
:105cdc00e24f51004b003200e44f510008003200fb
:105cec00e14f51002e00320041c1b3000a00780090
:105cfc0078f907004f0578004f04be00000006003d
:105d0c00c219de001b003200e48044000001eb00ed
:105d1c000201e800114490000884fb008004eb00b1
:105d2c00484bdd00c843de00870373004843dd00a9
:105d3c00214490008884fb000800200006044400e5
:105d4c0087844c001183fb008003eb0008044300a4
:105d5c0089844b0031439000c833dd0006002000dd
:105d6c00061a4400079a4c00e4804000830f51004f
:105d7c00e7ff390021c0b300414598008040eb009b
:105d8c00914298009a0090000a00780001000100ee
:105d9c004f0578004f04be0000000600d8ff370006
:105dac000300e000f3ff32000001eb0082804400ae
:105dbc00c1409000015a78000201e800830f5100a5
:105dcc0007003100ba04900082804400c14090006a
:105ddc00015a78000201e800830f5100f9ff3900e5
:105dec00ba02900021c0b300414598008040eb00fe
:105dfc00914298009a0090000a007800010001007e
:105e0c00e3ff37008301d100daff3200e480440065
:105e1c000001eb0091439000c83bdd001183fb00b7
:105e2c00069a43000201e8008180e800828f51004d
:105e3c00d0ff360091439000c83bdd001183fb007e
:105e4c00069a43000201e8008180e800828f51002d
:105e5c00f0ff3e00c7ff370040009000c1d7220082
:105e6c001108980061c822007100980081cf2200af
:105e7c0001089800000006004000900061e4220038
:085e8c00210898000000060047
:020000040000fa
:105e9400889fbe0091019000701a90008002eb0070
:105ea400e90f5200e08f5a0045013e00040601004c
:105eb400090037001c0037003c0037004f00370052
:105ec40080003700b4003700e300370018013700c2
:105ed4003d0137003c01370000c290000404e0009b
:105ee4000c00320020229000b0229000e00f5200fb
:105ef400e08f5a0005003a0014002000050020003d
:105f04002420980035209800020037001400200057
:105f140074189800501a90008491b900621898007f
:105f2400030178002b0137002002900060199000d3
:105f34006114b900611bb9000603540087835c0037
:105f44006124b900880f5300898f5b00020034007c
:105f540003014200080037000404ea00cfc4de0055
:105f6400880f5300898f5b0002003d0004815100bb
:105f74000100370006814100828f510015013a006b
:105f84006022b800242098003520980022002000c8
:105f940072189800200a9000400990000201420003
:105fa40022089800030178000a013700202290009b
:105fb400b022900060139000f0139000860f5200fe
:105fc400878f5a000600310061024200e0824a00d5
:105fd400242098003520980003017800fd00370044
:105fe40020c190000204e000f9003a0032002000d1
:105ff4007218980003017800f6003700d00a900068
:106004008009900003f0a7008301ea0003f0a700d1
:106014008381ea00700a9000830f52000a00340062
:1060240070039000800b9000a01190008591b9003e
:106034000299b9000201430083814b007200980069
:1060440003089800020037004200200072189800ec
:1060540060199000000a90008401780003f0a70002
:106064008381ea00d0129000858f5100d90034005a
:1060740040039000060252004013900006a3b900aa
:10608400483cdd004832de0004027400c8bade0079
:10609400b0119000611bb900860f5200878f5a001f
:1060a40006003c008301ea00611bb900860f520020
:1060b400878f5a00010035008401780003014100f4
:1060c400c4003700e00a90008009900003f0a700a4
:1060d4008301ea0003f0a7008381ea000012900024
:1060e400830f52000a00340070039000800b90006c
:1060f400a01190008591b9000299b90002014300f2
:1061040083814b0072009800030898000500370053
:106114006011b8002220980033209800520020001b
:106124007218980060199000000a900084017800a9
:1061340003f0a7008381ea00d0129000858f5100fc
:10614400a400340040039000060252004013900063
:1061540006a3b900c839dd004832de0004827100ac
:10616400c8bade00b0119000611bb900860f52005e
:10617400878f5a0006003c008301ea00611bb900c6
:10618400860f5200878f5a00010035008401780081
:10619400030141008f003700e0199000000b9000cc
:1061a4004001900002015300401390000693b9008f
:1061b400483cdd004832de0004027400c8bade0048
:1061c400301190006113b900860f5200878f5a0076
:1061d40006003c000201ea006113b900860f520078
:1061e400878f5a0001003500040178000301410043
:1061f40020229000b0229000001b9000901b900081
:10620400860f5200878f5a00050031006102420058
:10621400e0824a0024209800352098006d00370061
:10622400a0c190000304e0006a003a006022b800b4
:1062340024209800352098006300200073189800eb
:106244006112b900c022dd0004002000442098003f
:10625400552098005f00370040229000d022900023
:106264009648200006abb900483cdd004831de000a
:1062740002017400c8b9de000202520083825a008f
:10628400442098005520980085017800000b900068
:106294004001900002015300401390000693b9009e
:1062a4004839dd004832de0004027100c8bade005d
:1062b400301190006113b900860f5200878f5a0085
:1062c40006003c000201ea006113b900860f520087
:1062d400878f5a0001003500040178000301410052
:1062e40003f0a7008381ea0024082000848f510072
:1062f40004003c0013c0b30013c0980073002000d6
:1063040073189800b019900003f0a7008381ea0085
:10631400401a9000830f52002e00340013c0b300c3
:1063240013c09800730020007318980029003700e8
:10633400301a90000401780002f0a7000201ea007c
:1063440002f0a7000281ea00e90f510016003400b0
:106354000400e0000a003d00201b9000b01b9000e8
:1063640004a02100950020000602420087824a0012
:106374002418980035189800030178001500370098
:10638400201b9000b01b900004602e0065ff2f00be
:106394000602420087824a002418980035189800a3
:1063a400030178000b003700820020007218980067
:1063b4000001eb0032189800030178000500370053
:1063c40010012000dc0307000301780001003700fe
:1063d40003017800920098008040eb0021c09800ef
:0863e4004f04be00000006009a
:020000040000fa
:1063ec00b0009000e38f5000a800320004003e0083
:1063fc00e18f50004f00320090003e000a00370041
:10640c00e58f5000bc003200a7003900e68f500029
:10641c00c000320012c0b300e78f5000ce00320033
:10642c000041eb00cc003700f4f32f001161800029
:10643c0081026200e3c1200011322400d2bc2a0088
:10644c0026c220008209780081097800050b7800ab
:10645c00166280008602620026c420008209780041
:10646c0081097800050b7800156380000502620035
:10647c0026c620008209780081097800040b780078
:10648c00146180000490a00025c2200082097800cd
:10649c0081097800840a7800146180000480a000cf
:1064ac0026c220008209780081097800040b78004c
:1064bc00146280000490a00025c42000820978009a
:1064cc0081097800840a7800146280000480a0009e
:1064dc0026c420008209780081097800040b78001a
:1064ec00146380000490a00025c620008209780067
:1064fc0081097800840a7800146380000480a0006d
:10650c0026c620008209780081097800040b7800e7
:10651c00c12b2000410098005100980061009800a8
:10652c001100200071009800310098000041eb0030
:10653c0089003700f00090000041eb000100e00002
:10654c0085003a00f4f32f00116180008102620093
:10655c00e3c1200011322400d2bc2a0026c2200044
:10656c008209780081097800050b7800166280009a
:10657c008602620026c42000820978008109780016
:10658c00050b7800156380000502620026c620000a
:10659c008209780081097800040b7800146180006e
:1065ac000490a00025c2200082097800810978009f
:1065bc00840a7800146280000490a00026c4200095
:1065cc008209780081097800040b7800146380003c
:1065dc000490a00025c6200082097800810978006b
:1065ec00840a7800146180000480a10026c2200077
:1065fc008209780081097800040b7800146280000d
:10660c000480a10025c4200082097800810978004b
:10661c00840a7800146380000480a10026c6200040
:10662c008209780081097800040b78002100200091
:10663c00310098000041eb0047003700f00090005b
:10664c000041eb000100e00043003a002100200073
:10665c0071009800c000900082292000828f5000a9
:10666c00040036008100e900410098000041eb0075
:10667c0039003700410620007100980031002000dd
:10668c00310098000041eb0033003700f00090001f
:10669c000041eb000100e0002f003a004100200017
:1066ac00310098002c003700f00090000041eb0006
:1066bc000100e00028003a00210020007100980041
:1066cc00d000900082292000828f500004003600f8
:1066dc008100e900510098000041eb001e003700da
:1066ec0041062000710098005100200031009800f4
:1066fc000041eb0018003700f00090000041eb0067
:10670c000100e00014003a00610020003100980004
:10671c0011003700f00090000041eb000100e00098
:10672c000d003a002100200071009800e00090005c
:10673c0082292000828f5000040036008100e9007d
:10674c00610098000041eb0003003700710020004d
:10675c00310098000041eb00c000900031618800ce
:10676c00d002900035628800600390003663880088
:10677c00f00090000100e000020032008100e9000e
:0c678c0071009800024078000000060038
:020000040000fa
:1067980010250000ce02000080000000da11000081
:1067a8000200000080000000dc1100000200000070
:1067b80080000000fe2700000200000080000000aa
:1067c800de1100000200000080000000de2700004b
:1067d8002000000080000000e0110000020000001e
:1067e80082000000ffff00001a2a000002000000db
:1067f80080000000ec11000024130000800000005d
:10680800102a00000a00000080000000002a000092
:106818001000000080000000e611000002000000e7
:1068280082000000ffff0000e811000002000000e5
:106838008200000000100000001000001c01000091
:1068480080000000aa1100002a000000800000005b
:10685800ea1100000200000080000000d4110000ce
:1068680006000000800000007411000036000000df
:10687800800000001c11000058000000800000008b
:10688800002800000002000082000000000048000c
:10689800068c0c00c812f900181a1f0028251f00c2
:1068a8002bfb3000ba3656003cce41001c473f0057
:1068b8004c335100f55582005ad75e00f162cf0083
:1068c800666d6a00c96de20070b573004176840098
:1068d800787c7a00297c89007d9c7e00617fd800c5
:1068e8007fff7f00d87f61007f9c7e00897d290023
:1068f8007c7c7a008478410076b57300e270c90028
:106908006d6d6a00cf66f10062d75e00825af500ad
:10691800553351003f4c1c0047ce4100563cba004d
:1069280036fb30001f2b2800251a1f00f918c80055
:10693800128c0c004806000000b8f90074f3380007
:10694800ed07e700e6e0d800dae1d40005cf46001d
:10695800c9aac30032bee400b8c1b300cdae0b0073
:10696800aa7ea50029a10f009d31990093953700b3
:10697800921e8f004b8cbf00897c87008485d700ce
:106988008377820064819f0080288000018028002e
:10699800809f80006481770082d7830084857c0093
:1069a80087bf89004b8c1e008f379200939531006a
:1069b800990f9d0029a17e00a50baa00cdaec100ac
:1069c800b3e4b80032beaa00c346c90005cfe1004f
:1069d800d4d8da00e6e00700e738ed0074f3b80031
:1069e800f900000048068c000cc81200f9181a00bb
:1069f8001f2825001f2bfb0030ba3600563cce005e
:106a0800411c47003f4c330051f55500825ad700ce
:106a18005ef16200cf666d006ac96d00e270b50074
:106a28007341760084787c007a297c00897d9c00fb
:106a38007e617f00d87fff007f000000000000001b
:106a4800000000000000000000000000000000003e
:106a5800000000000000000000000000000000002e
:106a6800000000000000000000000000000000001e
:106a7800000000000000000000000000000000000e
:106a880000000000000000000000000000000000fe
:106a980000000000000000000000000000000000ee
:106aa80000000000000000000000000000000000de
:106ab80000000000000000000000000000000000ce
:106ac80000000000000000000000000000000000be
:106ad80000000000000000000000000000000000ae
:106ae800000000000000000000000000000000009e
:106af800000000000000000000000000000000008e
:106b0800000000000000000000000000000000007d
:106b1800000000000000000000000000000000006d
:106b2800000000000000000000000000000000005d
:0c6b380000000000000000000000000051
:020000040000fa
:106b440000082000620eb6000000e900cf00de005d
:106b540000508100e20f50001e00320005003e008c
:106b64000000e00008003200e10f500056003a0037
:106b740013003700e30f500044003200e40f5000cc
:106b840051003a00310037000104e00009003a00e6
:106b9400305081000000e0000300320060a02200b9
:106ba4001008e90048003700100020000050890058
:106bb40045003700800c2000305089004200370027
:106bc4000104e00040003200200020000050890051
:106bd4003d0037002250810070bb2000800f51001f
:106be4000a003e0040a022001008e8000104e00072
:106bf40035003a000008eb004006200030508900c0
:106c040040002000005089002f0037000104e000fc
:106c14000700320040a022000008eb0040062000dc
:106c240030508900300020000050890026003700d1
:106c340040a022000008eb004006200030508900ec
:106c440040002000005089001f00370030508100b0
:106c54000000e0000600320060a022001008e900f5
:106c640011c0b300640050000148780016003700da
:106c740020a022000048eb00800c20003050890046
:106c840000a022000008eb000f0037003050810004
:106c94000000e0000600320060a022001008e900b5
:106ca40011c0b300630050000148780006003700ab
:106cb40030a022000048eb00800c200030508900f6
:106cc40000a022000008eb0000042000620eb600c1
:106cd4000000e900cf00de0040508100e20f5000c8
:106ce4001e00320005003e000000e00008003200f3
:106cf400e10f500056003a0013003700e30f500034
:106d040044003200e40f500051003a0031003700d3
:106d14000104e00009003a00705081000000e00026
:106d240003003200e0a022001008e9004800370008
:106d3400100020004050890045003700800c2000de
:106d440070508900420037000104e0004000320026
:106d540020002000405089003d003700625081002f
:106d640070bb2000800f51000a003e00c0a022002a
:106d74001008e8000104e00035003a000008eb00c8
:106d840040062000705089004000200040508900d7
:106d94002f0037000104e00007003200c0a02200e9
:106da4000008eb00400620007050890030002000ed
:106db4004050890026003700c0a022000008eb00e4
:106dc4004006200070508900400020004050890097
:106dd4001f003700705081000000e0000600320000
:106de400e0a022001008e90011c0b30064005000c4
:106df4000148780016003700a0a022000048eb00ec
:106e0400800c20007050890080a022000008eb0054
:106e14000f003700705081000000e00006003200cf
:106e2400e0a022001008e90011c0b3006300500084
:106e34000148780006003700b0a022000048eb00ab
:106e4400800c20007050890080a022000008eb0014
:046e54000000060034
:020000040000fa
:106e5800889fbe0000047800383091000000e000f0
:106e680044003a0088b890007134980018309200b5
:106e7800e30f50003f003a0018d892000004e000e9
:106e88003c003200182892004823920058019100d3
:106e980080b3b90038009100000043006103b900d5
:106ea800610ab9000402530085825b006113b900ce
:106eb800860f5200878f5a000200340001004100fb
:106ec800080037000203ea00cfb3de00860f520045
:106ed800878f5a0002003d000280500001003700f1
:106ee8000480400040049900683191000200e000ed
:106ef80003003400e8019100f80491000200370013
:106f0800f8019100e804910018b990006103b900f4
:106f18006112b9000402530085825b00611bb9004d
:106f2800860f5200878f5a00020034000280410009
:106f3800080037000903ea00cfb3de00860f5200cd
:106f4800878f5a0002003d000900510001003700f8
:106f58000400410010bc9800420f200008014100c5
:106f6800e83291000882e800e839920082050700bb
:106f7800000ceb0018309200e10f50004d00360075
:106f880018289200682192008091b900180090009a
:106f9800800041003104980018289200582192007e
:106fa8008090b90018004000200498004004980020
:106fb80051049800781a9000d838920011a2b900ac
:106fc8000402420085824a00451498000501ea003f
:106fd800521498007a014400b8089000e8329100f1
:106fe80024042000080242008001eb00620507002b
:106ff8001820900030249800c82892000148a30067
:10700800180032000080b90000004000818048006c
:107018000100780000f0a7000080ea00d83892004c
:107028009100780054632400048ab90004024200e5
:1070380085824a0005a9b9000201410083814900ff
:107048008300780001f0a7008180ea0000805000ea
:107058002c040700501c98000000ea00601c9800ef
:107068000800370008219000583892001091b900a4
:107078000201410083814900531c98000300ea0083
:10708800601c9800c202200008014100c808900056
:1070980058009000e83291004404200008024200a1
:1070a8008001eb0034050700282090004024980058
:1070b8000c00370018289200882892008088b900b0
:1070c800a820900001004000402498001828920051
:1070d800f82092008088b9009820900001004000b4
:1070e80030249800d8399200620420000801410039
:1070f800f6004400c02720000800400093017800f3
:0c710800e20107004f04be00000006007a
:020000040000fa
:10711400889fbe008a9fbe008c9fbe00000478003a
:10712400080078004bff070020028000210e200099
:107134002102880038239000083a90001301c1000e
:10714400c8229000983b90001241c5000100cd0078
:10715400512498001301c6001201c0000200cd00a2
:1071640062249800200288000183d10040db2d00b6
:107174000281b80071249800068551000a2c9800f9
:107184000603ea0003035300162c9800282a9000f3
:107194000489b900c41add004c10de0000807200be
:1071a400302c980004d5b900c45cdd004c51de00dd
:1071b40002817400422c980004b3b900c43cdd0081
:1071c4004c32de000482740004037800542c9800ce
:1071d400820378008001780083007800040078003e
:1071e4001288e6000101fd001088e6000100fd00a0
:1071f4001090e6000200fd00610ab9004f81de0034
:1072040004004000850049008180d1000080d30043
:107214008000780001805100f3d12300940e2000f7
:1072240055952700008541001aa0e6000405780062
:107234004240ae0015d0e600050578006a2c98009f
:10724400818353000781410012a0e6000401780005
:107254004240ae001590e6000501780082037800f4
:10726400722c9800810053000183410016a0e600af
:10727400040378004240ae0015b0e6000503780030
:10728400063498006006200008004000c12b20004e
:1072940001d5b9000a0545008b854d000b0878001f
:1072a40001bab9000402420085824a0045349800bc
:1072b40001b2b9000402420085824a0055349800a4
:1072c4005838920090047800682a9000a0aa2a00f6
:1072d4000482b80052552500782890000096b80022
:1072e400083590000a91b800050378000d03530097
:1072f40003025300d23c29000090b8000a95b8005c
:10730400010178000b01510009a2b90004024200f6
:1073140085824a00153498000991b90002014100a0
:1073240083814900233498004f06be004f05be00f8
:087334004f04be00000006003a
:020000040000fa
:10733c00c3e8a900000000000000000009a1220021
:10734c00800c78000000eb009004980011c0b30092
:10735c00914c9800e044980060c0b300804c9800b9
:10736c00f3f32f001061800000826100e2c1200065
:10737c0010322400d1bc2a0025c22000010978005b
:10738c0000097800840a780015628000058261008b
:10739c0025c420000109780000097800840a7800cf
:1073ac00146380008481610025c6200001097800e7
:1073bc0000097800830a7800136180000390a00014
:1073cc0024c220000109780000097800030a780023
:1073dc00136180000380a00025c220000109780001
:1073ec0000097800830a7800136280000390a000e3
:1073fc0024c420000109780000097800030a7800f1
:10740c00136280000380a00025c4200001097800cd
:10741c0000097800830a7800136380000390a000b1
:10742c0024c620000109780000097800030a7800be
:10743c00136380000380a00025c62000010978009a
:10744c0000097800830a78000060fe004c062000da
:10745c006aae2a000b002000090078000104070026
:10746c000028a3000200320034cea800010037002f
:10747c0034cea9000038a3000200320034aea800bc
:10748c000100370034aea9000c0478000060fe0047
:10749c000a00be00580807000060fe000a00be008b
:1074ac00550807000060fe000a00be0052080700e5
:1074bc000060fe000a00be004f0807000060fe00de
:1074cc000a00be004c0807000060fe000a00be0067
:1074dc00490807000060fe000a00be0046080700cd
:1074ec000060fe000a00be00430807000060fe00ba
:1074fc000a00be00400807000060fe000a00be0043
:10750c003d0807006a045400e0ff3a00d2ff370040
:020000040000fa
:10751c000000060000000600000005000280fb00d1
:10752c000000ea004f00de0000000600000005002d
:10753c0080407800f0c7b30002c8b30082cf50007f
:10754c00030032000100fb0000f0a7000000ea007d
:10755c000000060080007800f0ff270002002800e1
:10756c00828f5000030032000100780000f0a70069
:10757c000000ea0000000600f2ff2f00f3ff2700d6
:10758c000400200005002800840f5000858f58004f
:10759c00040032000001be00e00f5000e08f5800e4
:1075ac00020035000200be00000006006001100061
:1075bc00e08118000200be0000000600fbff37004f
:1075cc006022b80006002000070028000400e1003b
:1075dc000588e1000690e1000798e10014003200f4
:1075ec000203be000002be00e00f5000e08f580006
:1075fc00e00f5900e08f5900030035000400be0075
:10760c000601be00000006006000b8006011b80062
:10761c0004025000858258000603590087835900e4
:10762c000400be000601be0000000600f6ff370095
:10763c00f4ff2f00f5ff2f00f6ff2f00f7ff2700b8
:10764c000400be000601be0000000600eeff37007d
:10765c00889fbe000004be006011b800bfe40700a4
:10766c000000e00001003d0009f0a2008801780054
:10767c000901780003007800820078004f04be00f6
:10768c0000000600889fbe008a9fbe000004be005a
:10769c000205be006022b8006033b800a5e4070004
:1076ac000000e00001003d000bf0a2008803780010
:1076bc00090378008a0278000b0278000700780032
:1076cc008600780005017800840178004f05be0023
:0876dc004f04be00000006008f
:020000040000fa
:1076e400881f78000004780018309000a8309000bb
:1076f40000b4980011b4980018089000a8089000ed
:1077040020b4980031b49800010e20008880400015
:1077140040072000080040000ef70700b8a89000ba
:1077240071b498007888900000bc9800710c99009e
:1077340000149900482892000018a3001000320099
:10774400782892000000e00003003a00e828920044
:10775400712c9a0003003700782892000000e90099
:10776400702c9a0078299200883092000000eb0077
:10777400810f510020003100582892001e0037006c
:1077840068319100801120000800400088007800d2
:10779400bff9070038289100e60f500011003e00a1
:1077a40058129100e812910058199100c8109100e4
:1077b4000191b9000201420083814a0052149900e8
:1077c4006314990068119100683090000000510022
:1077d400f8b19000030151007224990011bc980083
:1077e40005003700f820910078b090000080400038
:1077f400e830900001005000e83090000080400024
:107804006034980038289100e40f50000a003e00cc
:1078140031002000810f50001600310011002000bb
:107824000000e0001300320021002000810f50000e
:1078340008003a000f00370051002000e70f500005
:107844000c003200e80f50000a003200810f500093
:10785400020032008000eb00060037004828920046
:10786400410020000058a3000200320010c0b30001
:1078740020dc9a0041b498001800900050b498009d
:10788400e830910061b498004f04780000000600cd
:020000040000fa
:10789400889fbe00030378009100900001027800e5
:1078a40004f0a7000402ea0004f0a7000482ea003e
:1078b400d0019000830f520004003500e0019000d5
:1078c4000310a0006300980003003700e00190005b
:1078d4000310a1006300980001f0a7008100ea00f2
:1078e40001f0a7008180ea00c0019000838f50005e
:1078f40004003d00e00090000100a0006100980039
:1079040003003700e00090000100a100610098002e
:107914001204780008c4b9000804440089844c00a7
:107924008900780001f0a7008180ea00120290002b
:1079340004a2b9000402420085824a0005017800cd
:1079440002f0a7000281ea008100410006b2b900fa
:107954000402420085824a00050278002003900058
:1079640005b3b9000603430087834b00878f50009b
:1079740004003900300190000210a0003200980089
:1079840003003700300190000210a100320098007b
:10799400100190000491b900020241008382490061
:1079a400858f500004003100b00090000100a00059
:1079b4003100980003003700b00090000100a100de
:1079c4003100980090017800b0009000e3806000de
:1079d4000041eb0001003a0061c1610060029000c7
:1079e400630262008040eb0002003a008300d10091
:1079f400e1c060000204e000060032001200200032
:107a04000104e00001003200320020000208780086
:107a1400050037000001eb000104e0000100320022
:107a240022002000020878004f04be000000060077
:020000040000fa
:107a3400889fbe00000478008004eb00293499007c
:107a440060ee26000100200050849a0061849a00b0
:107a54003000200010349a0029349a006026200057
:107a64000800400009487800202b2000080040004e
:107a740091070700c3fe2f0020618000008261008f
:107a84001401b300e2c1200010322400d1bc2a004a
:107a940045c220000109780000097800840a7800b2
:107aa40025628000058261001401b30045c42000f2
:107ab4000109780000097800840a780024638000b2
:107ac400848161001301b30045c6200001097800d8
:107ad40000097800830a7800002b20000800400089
:107ae40009487800789092000000e00002003a0013
:107af4001000200070949a008044eb0009ec9a0076
:107b040000c1b30000fc9a0019fc9a004024200034
:107b1400080040002d06070000d0270050049900fb
:107b2400f0002000600499002000200070049900f7
:107b3400683091006011b800321499004314990020
:107b440078109100cf80de00c000dd00000020002e
:107b540050149900611499000000eb00302c990036
:107b6400622c9900732c990010dc9a0009dc9a00ad
:107b740029dc9a0040002000600c9900e0172000e6
:107b840008004000b3050700e02220000800400080
:107b94000948780000232000080040000907070076
:107ba4006023200008004000160707000800780042
:107bb400a00707004001200070949a007207070094
:087bc4004f04be0000000600a2
:020000040000fa
:107bcc00881f78000004780020028000210e20001d
:107bdc002102880068029000140c9800759e240005
:107bec001301c000780390001201c4001201c400fc
:107bfc000500cd00250c9800200288002002800092
:107c0c0021028800083b90001301c100983b9000b2
:107c1c001201c5000100cd00310c98001301c40005
:107c2c001241c2000100cd00410c980020028800d6
:107c3c0008007800a8fe07006831900000082000ba
:107c4c000201b80003007800820078000100e00017
:107c5c0010003a00800040000280220081004100a8
:107c6c0091007800113c98000002b000f107200050
:107c7c00810f5000010036000008b10000004000e8
:107c8c00018022000080400010007800003c980029
:107c9c0025003700000140000380220002814100d2
:107cac00120178000000e800f3072000830f500059
:107cbc00010036000008b100800140000480220061
:107ccc008301420013021100048ab800050141002f
:107cdc00123c98007f004000f2072000820f5000f9
:107cec00010036000008b1000001400003802200b2
:107cfc0002814100120178000000e800f307200027
:107d0c00830f5000010036000008b1000000400055
:107d1c000380220000804100100011000088b80090
:107d2c0001014100023c98004f047800000006005d
:020000040000fa
:107d3c00118f80008100e800118f880011009800dd
:107d4c007c050700e2050700c12b2000416188007b
:107d5c004162880041638800216088003000200067
:107d6c005061880060618800506288006062880001
:107d7c0050638800606388005000200030618800e8
:107d8c00306288003063880091618800214ca80023
:107d9c00f3f32f001061800000826100e2c120002b
:107dac0010322400d1bc2a0025c220000109780021
:107dbc0000097800840a7800156280000582610051
:107dcc0025c420000109780000097800840a780095
:107ddc00146380008481610025c6200001097800ad
:107dec0000097800830a7800136180000390a000da
:107dfc0024c220000109780000097800030a7800e9
:107e0c00136180000380a00025c2200001097800c6
:107e1c0000097800830a7800136280000390a000a8
:107e2c0024c420000109780000097800030a7800b6
:107e3c00136280000380a00025c420000109780093
:107e4c0000097800830a7800136380000390a00077
:107e5c0024c620000109780000097800030a780084
:107e6c00136380000380a00025c620000109780060
:107e7c0000097800830a780021e3a800e5060700d2
:047e8c0000000600ec
:020000040000fa
:107e9000042eef00142eef00242eef00342eef00fe
:107ea000442eef00542eef00642eef0030f9210035
:107eb00000708800f03f200080708800f08f2b0059
:107ec00000718800302eef0000002f000072880043
:107ed0001100200081728800013c2000017388009d
:107ee0000c2eef001c2eef002c2eef003c2eef008e
:107ef0004c2eef005c2eef006c2eef000a2eef00f0
:107f00001a2eef002a2eef003a2eef004a2eef0035
:107f10005a2eef006a2eef00062eef00162eef000d
:107f2000262eef00362eef00462eef00562eef00e5
:107f3000662eef003181210071708800f110200061
:107f4000f170880071802000717188007072880063
:107f5000f20b2000103a8000000161006004200054
:107f60007105200023742000804978008149780041
:107f70008249780002f82f002436800084016100d5
:107f80005303b30023368800f30f2c0075348000b0
:107f9000058261000480a00074348800643480008d
:107fa0008481610004d022000302720064348800de
:107fb000c5358000050161004202b300c23588006a
:107fc000123a80000260a0002374200080497800eb
:0c7fd0008149780082497800000006001a
:020000040000fa
:107fdc00022cef00100020002060880080002000a0
:107fec00306088000a2cef001a2cef001e2cef00da
:107ffc0040202100006188004020200000628800a1
:10800c000063880013002c00e2c120001032240011
:10801c00d1bc2a0024c22000010978000009780094
:10802c00030a780024c420000109780000097800b4
:10803c00030a780024c620000109780000097800a2
:10804c00030a7800c30f200044c220000109780005
:10805c0000097800030a780044c420000109780064
:10806c0000097800030a780044c620000109780052
:10807c0000097800030a7800262cef00462cef004c
:10808c00662cef00282cef00482cef00682cef003a
:10809c002a2cef004a2cef006a2cef002c2cef005e
:1080ac004c2cef006c2cef00322cef00522cef001c
:1080bc00722cef00342cef00542cef00742cef00da
:1080cc003a2cef005a2cef007a2cef003c2cef00ee
:1080dc005c2cef007c2cef003e2cef005e2cef00b4
:1080ec007e2cef0080d624005b0607000728a90031
:1080fc002728a80010b020000060880000000600af
:020000040000fa
:10810c00800378000000eb001700e6000000000080
:10811c000000000000000000889fbe008781cf0097
:10812c00e28051000139dd0000002800800251007e
:10813c0005027800c12add000600240006a3b90060
:10814c0005a4b90000002f000981b9000603410005
:10815c008783490005ccb900008020000981b90053
:10816c00060341008783490005ccb90000b02f00fd
:10817c000981b900060341008783490005ccb90089
:10818c00003820000981b9000603410087834900ab
:10819c0005ccb90000d62f000981b90006034100b7
:1081ac008783490005ccb900002120000981b90062
:1081bc00060341008783490005ccb90030e52f0048
:1081cc000981b90006034100878349004f33de0063
:1081dc004138dd0000037300cfbbde000000280037
:1081ec0006034000e0834b004109de0070001100e3
:1081fc000233de000038dd000003730082bbde00ba
:10820c000100a3000500390024a8250004b0b90022
:10821c004f00de00c108dd0001037000060078008d
:08822c004f04be000000060033
:020000040000fa
:1082340001407800818d800001040100708d800070
:1082440000040100608d800000040100508d800056
:1082540000040100889fbe008a1f78000004be004d
:10826400e3020700801c2100eb03070013c0b300e6
:1082740000c1eb00c1012100201b21003cf20700da
:108284002a1b21000a0078001af007000a0078006f
:1082940022f007000a007800f1f607000a007800cf
:1082a400f7f607000a007800e3020700811c2100aa
:1082b4000a007800e5030700408f800011002000c9
:1082c40031009800c8050700408f8000815c2800b9
:1082d40011009800015e280001087800a011240014
:1082e400408e880000122400508e88004012240022
:1082f400608e880080122400708e88000800be0002
:108304008d0507004f0578004f04be0000000600ed
:10831400201b2100918d8000010401008a05370093
:10832400808d8800718d8800628d8800538d88004f
:1083340000000600a11124000108780001122400a5
:108344001100980041122400210098008112240099
:08835400310098000000060052
:020000040000fa
:10835c008000780022188000e2009800101880003d
:10836c00c18a920082825200718a920000005200ef
:10837c002189920002a9b900318b92000683b900c1
:10838c000603410087834900413add004f31de008e
:10839c0002017200e20098005189920002a9b90012
:1083ac00618a92000482b90004024100858249006e
:1083bc004128dd004f21de0002017000f200980020
:1083cc00210891000000e00004003a0000002800a1
:1083dc000003b400b0089900060037000000e0006c
:1083ec000400320051399200000028000003b40050
:1083fc000009d100412892000008a30008003a00af
:10840c00513a9100310891000482b800613b91000f
:10841c0061309100050143008091b900b2009900d0
:10842c00210891000000e00007003a001000200035
:10843c00a008990000fe2f002803b600a000b3008e
:10844c0040198800060037000000eb00a0089900d6
:10845c0000fe2f002803b600d000b300401988009e
:04846c000000060006
:020000040000fa
:10847000f04090008140e800714098007041900009
:1084800080489000814f5100020039008040eb008d
:1084900071409800904890000104e0002b003200e9
:1084a000f04090000104e0001b003a00e040900022
:1084b0000104e00004003200e04090008140e90047
:1084c0006140980014003700900090000100e00027
:1084d00005003a0031c0b300614098009000780078
:1084e000110098000c00370090009000e3806000bd
:1084f00006003a0011c0b30061409800900090005f
:10850000c208de00110098000300370090009000c0
:108510008100e90011009800604190008000eb00ac
:108520000204e00014003a007041900000489000fe
:108530000080fb000000d100c1002000804f5100ee
:108540000d0039008000eb000b003700f041900077
:10855000404190004100200082cf510001003900cd
:108560008000eb007041900050409000804f51001f
:10857000010031000130a000010078000000060079
:020000040000fa
:10858000889fbe008a9fbe002b028000270f20001c
:108590002602800086836300270eb300270288002e
:1085a0000000ca000180ca000030cb000a00cd00e4
:1085b00012047800920490000980ca0048018800e3
:1085c000220490008a037800080378001301c60093
:1085d000d20390008703ea000700c8000000cb0028
:1085e0000800cd00f2039000820c9000870f540029
:1085f00004003c0088037800890f540001003d000e
:1086000089037800070a78000300e0000d003200bb
:108610000500e0000500350013c0b300810f5000d5
:10862000060034008041eb000400370013c0b300a3
:10863000810f500001003d008041eb000304e00089
:108640000d003200320290008a0278001301c0004f
:10865000620090000000ea000000c8000702540019
:10866000c20390001241c2000000cb001001800044
:10867000210180000089be002b0288004f05be004a
:088680004f04be0000000600db
:020000040000fa
:10868800a0309100e58f50001b003200a03091000f
:1086980003c1b30012c0b300e28f50000e003200d5
:1086a80004003e008041eb00e18f500008003a00d2
:1086b8000900370003c1b300f2c0b300e38f5000d4
:1086c800050032008041eb00e48f500002003200c8
:1086d8008041eb0003417800d03091000148a300ad
:1086e8000300320042f09a0053f09a00020037006b
:1086f80043f09a0052f09a00a03092000100e00086
:1087080014003200a0309200e28f500006003200c0
:10871800e38f500007003200e18f50000b003a0051
:1087280001e89a00090037008040eb0001e89a0050
:10873800060037008040eb0001e89a00612620001f
:108748008080400012c0b300824878008000eb00af
:0887580021309a000000060028
:020000040000fa
:10876000b0009000e18f5000100032000600390088
:10877000e28f50001e00320032002000828f500035
:1087800027003a0027003700c00090000001eb00ee
:108790000108a30023003200d00090000100a000d7
:1087a00051009800120020001e003700c000900009
:1087b000120020000118a3001a0032009000780077
:1087c0000100e00005003a00d00090000110a00078
:1087d0005100980032002000120037000108e90023
:1087e0008000eb0011009800220020000d003700ef
:1087f000900090008100e80011009800a001900016
:1088000022002000838f500006003900d000900025
:108810000100a100510098000001eb0001003700a9
:108820000001eb008000eb0041009800320098004e
:04883000000006003e
:020000040000fa
:10883400881f780000047800b8009000f07c2000c5
:10884400808f50002b0036000000eb0030049800ad
:108854007b0407000004e000040032001880fb00e1
:108864000000e9004f00de00004c78001800900082
:108874000048a30004003200180090000050a0003b
:108884001004980003003700180090000050a10065
:10889400100498006d0407000004e0000900320091
:1088a400180090000040a200100498009800900066
:1088b400100020000148a300010032000080eb00fa
:1088c4002004980068004400e8fe07000028a30084
:1088d4000200320034cea8000100370034cea900d3
:1088e4000038a3000200320034aea80001003700b3
:0c88f40034aea9004f047800000006001c
:020000040000fa
:1089000060029000d0019000830f520028003100d7
:108910001003780092017800052020008382420035
:1089200004402000848f520008003e001002900096
:10893000a0029000c619dd00069bb90006034200a4
:1089400087834a001600980027009800900278005c
:108950001201900004202000020242000340200087
:10896000830f520008003e0030039000c0039000c7
:108970004611dd000591b9000201430083814b00df
:108980003200980043009800200190004691de00dc
:10899000a2009800400190004691de00d2009800ad
:1089a000e00090008100e8006100980002003700bc
:0c89b00011c0b300015098000000060048
:020000040000fa
:1089bc005417220074089800431e200003109800de
:1089cc008000eb002110980031109800f2ff270076
:1089dc0012109800759e24004510980096612b008b
:1089ec0056109800751898000418980013189800e1
:1089fc00311898004118980022189800c24f250091
:108a0c005218980043b02a0063189800022098006e
:108a1c00923db00042b898008200200052b89800f5
:108a2c0071b898000100990061b89800a18b2200e0
:108a3c001100990061742d002100990000000600be
:020000040000fa
:108a4c00881f780000047800513c9a006000b80040
:108a5c00500c9800610c98006014980071149800e8
:108a6c0020bc980031bc98000000eb00102498004a
:108a7c0020249800000c780010049800100c990029
:108a8c00200c99008011200008004000970007007e
:108a9c004129200088804000002a20000800400066
:108aac006a020700f2ff27000000210011000900f4
:108abc000200d900202c9800c0272000080040009c
:108acc005e03070010c0b3004f04780000000600de
:020000040000fa
:108adc00881f7800207d220095fc0700207c220056
:108aec00a200070080672200ec010700207522001d
:108afc00c5030700e068220049010700007422004a
:108b0c002e030700607422003c0307000051220072
:108b1c00c5fb0700807d2200a10307008801070028
:108b2c0040a7a800e431ef0000512200a0ff07008d
:108b3c00217d220000512200c1ff07000044780073
:108b4c000804e00002003200207d2200df02070052
:0c8b5c00084078004f047800000006007c
:020000040000fa
:108b680011662500410098003100980041ba2100a3
:108b780021009800c1042500610098005100980068
:108b88006011b80032089800430898008000eb0094
:108b98002128980061089800121098002310980066
:108ba80032109800431098005128980061289800c6
:108bb800c211200002089800028e2000720098005e
:108bc800f24a200012089800c22e200022089800bd
:108bd800a21a2000020878001100980011309800ad
:088be80051089800000006008e
:020000040000fa
:108bf00000102300203a88004827ef004e27ef009e
:108c000040042000303a88006027ef006227ef0020
:108c10006427ef006627ef006a27ef006c27ef005c
:108c2000a1092000320020008007200033742000ba
:108c300080497800814978008249780071052000d8
:108c40001200200060042000237420008049780076
:108c500081497800824978004207ab00feff3a0064
:108c600001022000123a800002806000fdff320005
:048c700000000600fa
:020000040000fa
:108c7400e20f50000d003200e30f500014003200e8
:108c8400e10f50001a003a00c0ff2f00240cb60078
:108c9400d2bc2a0011322400e3c1200082097800ea
:108ca400810978002061880011003700c0ff2f007f
:108cb400440cb600d2bc2a0011322400e3c12000c7
:108cc4008209780081097800206288000800370052
:108cd400c0ff2f00640cb600d2bc2a00113224005d
:108ce400e3c12000820978008109780020638800ac
:048cf4000000060076
:020000040000fa
:108cf80001b0200071089800113b21000110980074
:108d0800618e200051089800d1c7220061089800a0
:108d18006011b8006210980073109800021898004b
:108d280013189800b1aa2e00310898005155210057
:108d380041089800c1712000411898003131b000f5
:108d4800511898004135200011109800110020009a
:108d5800211098008000eb00311098008117200046
:108d680041109800017e2000511098000000060074
:020000040000fa
:108d7800889fbe0000047800004ceb000000eb0068
:108d88001004980020049800f002070019c0b300ee
:108d9800b30207000004e000fdff32001804e00001
:108da80006003a004103070010049800e40f500041
:108db8000a003a00094c7800020037003d0307001a
:108dc8001004980018009000e40f500003003a00c7
:108dd800080307004f04be0000000600e10f500022
:0c8de800ebff3a005002200052f9070097
:020000040000fa
:108df400408f80008000eb0001087800110098008b
:108e04002100980031009800410098006011b800da
:108e140052009800630098007100980001089800bf
:108e2400110898002108980031089800410898001a
:108e34005108980000000600418f800071019000e5
:108e4400e10f51000100360000000600710190009e
:108e5400e80141008381410083814000800978005a
:0c8e64000201e800f20098000000060087
:020000040000fa
:108e7000881f7800287d2200806722006dfe070091
:108e80000051220000fe0700e431ef00c80090000e
:108e9000601a2d00808f50000e003a0038009000bc
:108ea0000008a3000b00320000000000feff3700a6
:108eb000380090000028a30001003200ef020700f4
:108ec000f8020700207c22003e0007004f047800d3
:108ed00000000600c8009000601a2d00808f50002e
:088ee000f7ff3a00f2ff370032
:020000040000fa
:108ee8008000eb0071b09800613098001100980084
:108ef800010878004100990011b89800603191008c
:108f08006011b80032109900431099007012910056
:108f1800cfa2de00c022dd0004002000541099001a
:108f280065109900312899006228990073289900e2
:108f380011d89a0021d89a004100200061089900b0
:108f480011c0b30001d89a004007b000e002070042
:048f5800000006000f
:020000040000fa
:108f5c00881f7800000478000023200008004000df
:108f6c00880078005f000700e02220000800400025
:108f7c001004e0000e003200e01720000800400052
:108f8c008800780003ef0700482892000038a300ff
:108f9c0007003a00c8109200381092000080600060
:108fac0003003200781892000000a000701c9a0098
:088fbc004f04780000000600dc
:020000040000fa
:108fc400881f78000004780028009000f30f5000f8
:108fd400130036000000eb00200498001804e000a1
:108fe40007003a00b202070010049800e40f500092
:108ff40005003a0010c0b300004c780002003700ae
:10900400ad02070010049800cdf607001800900088
:10901400e10f500002003a0060022000c6f8070089
:089024004f0478000000060073
:020000040000fa
:10902c00881f7800000478006e0044004701070098
:10903c0080042000080040007d010700e0062000ad
:10904c00080040008e010700c00520000800400009
:10905c00810107000008200008004000c70007003d
:10906c000000eb0040949800f1fe2f005194980002
:10907c006094980040062000709498004f0478008b
:04908c0000000600da
:020000040000fa
:1090900080017800c32892000128a3000c003a0048
:1090a000d33892001101780001002100810f510096
:1090b0000500340001027800110009000220d900e7
:1090c0000001780001003700f2ff2700a229980074
:1090d000b33091008100e800b1319900f38f500066
:1090e000020036008000eb00b1319900000006005c
:020000040000fa
:1090f000032b2000818141000001eb001304e000fc
:109100000a003200513992009201780012002000ca
:10911000908f510001003c000001eb001002900014
:10912000848f510001003d000210a000f1909200d8
:109130000100e00003003a00200ce20001003d00c5
:0c9140000220a0002200980000000600a1
:020000040000fa
:10914c00013a80000100e0000f0035001002200001
:10915c0001e8a3000d003a000000e8000198a3000c
:10916c000a003a000148a3000a0032000080e8001f
:10917c00f1702200228f8000810f510003003e000d
:10918c000000e90001003700000220004027ef003a
:0c919c0067f807004027ef000000060005
:020000040000fa
:1091a8006011b80012009800230098008000eb00be
:1091b80031009800520098006300980071009800f0
:1091c800120898002308980031089800520898005f
:1091d80063089800710898002210980033109800ce
:1091e80011109800621098007310980051109800a0
:0c91f800121898002318980000000600d0
:020000040000fa
:109204000000060000000500000005000000050045
:1092140000000500000006002190240001087800e9
:1092240041902400110098006190240021009800ce
:109234008190240031009800a190240041009800fe
:10924400c1902400510098000000060051009800cd
:049254000000060010
:020000040000fa
:10925800881f7800000478006e004400d0ff0700e3
:1092680080042000080040006d010700c0052000b0
:1092780008004000a3010700000820000800400083
:109288002e010700e006200008004000a3010700a7
:109298000000eb00409498004f047800000006009e
:020000040000fa
:1092a8000048eb008000eb003100980011009800a6
:1092b8007148980002c1b3000250980011509800fc
:1092c800614898004148980051489800510098001a
:1092d8001100200021009800411a2400110898006c
:0c92e800113b2100210898000000060046
:020000040000fa
:1092f40014ed230004a2b9000402420085824a004e
:109304008500780001f0a7008180ea000108780058
:109314003428240004a2b9000402420085824a00d1
:109324008500780001f0a7008180ea001100980010
:0c9334008000eb00210098000000060003
:020000040000fa
:10934000500ea80000f82f00f23580008200600067
:109350000106b300f135880020cea800f20f2800e6
:10936000e13580000101610001602300828070000e
:10937000e1358800010ea800bc06b6008001b300ec
:08938000e03588000000060042
:020000040000fa
:10938800918f210031089800917c260001109800e7
:1093980061752c0011109800a1f924002110980083
:1093a8002122220021089800529124000300200065
:1093b800020898001308980042009800530098008b
:0893c800de00070000000600b2
:020000040000fa
:1093d0008000eb0031009800410098005100980097
:1093e0006100980021009800710098006011b80099
:1093f0000208980013089800210898003108980086
:10940000410898001200200062089800316098001e
:049410000000060052
:020000040000fa
:10941400e18f500004003a00002092000000d100c7
:10942400614060000a003700002192001100200012
:109434000218a30005003a00a018920001f0a7004a
:109444008100ea008100ea00cf08de0001407800d4
:04945400000006000e
:020000040000fa
:1094580003002400830878000001eb0092009800c4
:10946800b2009800c300980062009800010820002c
:10947800510098006011b80012009800230098006d
:10948800320098004300980001002c000108780081
:0494980000000600ca
:020000040000fa
:10949c007cfa070084000700d2fd0700af0007002c
:1094ac0039000700cafa0700450007000e01070043
:1094bc00c3e8a8000000000000000000200f2000fe
:1094cc004400b6000050a0002002880000000600f6
:020000040000fa
:1094dc000000eb000050890021a022008048780099
:1094ec008100e800804878002050890030508900c5
:1094fc0040508900e7804000804878008100e800f7
:10950c008048780060508900705089000000060087
:020000040000fa
:10951c0070a1900080a99000723899000380990086
:10952c0010899000a08990001280990023809900e6
:10953c0020919000b0919000328099004380990066
:0c954c00f0899000538099000000060098
:020000040000fa
:109558007206200002087800a1142000410098003b
:10956800020898004108980041082000011098005e
:1095780041109800e20320000300200032189800f0
:0c9588004318980006ff070000000600d2
:020000040000fa
:10959400c03620000019880000202000101988001f
:1095a40060002000201988002823ef002e23ef00fc
:1095b4003023ef003223ef002623ef0060d624008f
:0895c40025010700000006006c
:020000040000fa
:1095cc000621ef0020112000600888000003200015
:1095dc0080088800de11e20002003a00a0d62400c8
:1095ec00e300070000e8a90020e8a800e07f2200c3
:0895fc000048eb00000006002e
:020000040000fa
:10960400f03fb1000180b10006003500ee0309000f
:1096140000000000403fb1000180b100fbff3d00ad
:109624001000b000203fb0000200350000800900a7
:08963400000000000000060028
:020000040000fa
:10963c001102200001087800c1c7220041009800e7
:10964c00e20d200003002000020898001308980087
:08965c00720007000000060087
:020000040000fa
:10966400e29c270003002000720098000308980081
:10967400320098004300980041002000010878005f
:08968400a10007000000060030
:020000040000fa
:10968c00e1682000010878005291240003002000ba
:10969c00720098000308980032009800430098006c
:0896ac009d000700000006000c
:020000040000fa
:1096b400f0f82f005c08b6000060a000e0428800cb
:1096c400f0ff28004208b60000e0a0001042880025
:0496d400000006008c
:020000040000fa
:1096d800350ea800200220000080090000000000cc
:1096e800350ea90001eca80001a8a90021a8a8002e
:0496f8000000060068
:020000040000fa
:1096fc0023d4240062d42400a1d42400e0d4240078
:10970c0005fb070041322100c01e2100cffa0700e3
:04971c000000060043
:020000040000fa
:10972000010878008000eb001100980012c0b3001f
:10973000124898006140980061c0b3000148980049
:04974000000006001f
:020000040000fa
:109744008000eb0001087800110098006011b80057
:10975400620098007300980022009800330098007b
:0497640000000600fb
:020000040000fa
:1097680080002000001188002222ef0070092000ec
:109778004011880021e2a8002342a800000006004a
:020000040000fa
:109788000000eb002322ab0004003a000040200058
:109798002202b6000000ea004f00de0000000600ca
:020000040000fa
:1097a8001000fa000000eb0080bf9f00fcff0700dc
:1097b8008fb89700010040000080fa000000060002
:020000040000fa
:1097c800881f78000004780008007800640007000b
:1097d80008007800930007004f0478000000060096
:020000040000fa
:1097e80021002000010878008000eb00110098009b
:1097f80031009800410098005100980000000600d0
:020000040000fa
:10980800881f78000004780008007800f4ff07003b
:1098180000352c00200498004f0478000000060052
:020000040000fa
:109828006011b80012009800230098008000eb0037
:10983800310098006200980073009800000006004c
:020000040000fa
:10984800881f7800000478000880e800a7fe070059
:10985800680044001e0007004f047800000006005e
:020000040000fa
:10986800e07f2200104078000004e000020032008f
:0c987800e17f22008048eb0000000600a9
:020000040000fa
:109884002202ab00feff32002222ab0001003200b4
:0c9894002222a900301180000000060014
:020000040000fa
:1098a000022020001311800083006100fdff3a00b8
:0c98b0000080fb00201188000000060072
:020000040000fa
:1098bc008000eb0041009800510098006100980076
:0c98cc00710098003100980000000600b8
:020000040000fa
:1098d800b1782200010878008127b00011009800b3
:0c98e8008000eb0021009800000006004a
:020000040000fa
:1098f4000021ef0002a1ef000421ef00a0a122004b
:089904000048eb000000060022
:020000040000fa
:10990c006011b80052009800630098001200980093
:08991c00230098000000060082
:020000040000fa
:109924006011b8005200980063009800120098007b
:0899340023009800000006006a
:020000040000fa
:10993c000101780080007800c011210095de37000d
:08994c00c0112100d1de37003b
:020000040000fa
:10995400e07f22000048eb0020e8a80011e1a80005
:0499640000000600f9
:020000040000fa
:109968009143270001087800d15f21001100980079
:0499780000000600e5
:020000040000fa
:10997c0020e8a900f08e880020e8a800000006006e
:020000040000fa
:10998c00a0a122000048eb0005e1a80000000600a1
:020000040000fa
:10999c00bffe07004efc070032fd0700feff37003c
:020000040000fa
:1099ac008000eb0001087800110098000000060010
:020000040000fa
:1099bc002024b00011c0b30001487800000006005c
:020000040000fa
:1099cc00b00090008100e800310098000000060013
:020000040000fa
:1099dc00a00090008100e800210098000000060023
:020000040000fa
:1099ec0021089800815e28003108980000000600cc
:020000040000fa
:0c99fc0011e1a90020e8a900000006000d
:020000040000fa
:0c9a0800101180006100600000000600ea
:020000040000fa
:0c9a140011c0b3000148780000000600fb
:020000040000fa
:0c9a200051ff070035ff070000000600a2
:020000040000fa
:0c9a2c008000eb00210098000000060004
:020000040000fa
:0c9a38004007b0004afc070000000600d8
:020000040000fa
:0c9a440020a02200104078000000060066
:020000040000fa
:0c9a5000a0a022001040780000000600da
:020000040000fa
:089a5c00d08e88000000060016
:020000040000fa
:089a6400e08e880000000600fe
:020000040000fa
:089a6c00008f8800ffff3700a6
:020000040000fa
:089a740000088000000006005c
:020000040000fa
:089a7c004aff0700000006008c
:020000040000fa
:089a840040ff0700000006008e
:020000040000fa
:089a8c00deff070000000600e8
:020000040000fa
:089a94007bff07000000060043
:020000040000fa
:089a9c0080ff07000000060036
:020000040000fa
:089aa4001bfa07000000060098
:020000040000fa
:089aac001cfa0700000006008f
:020000040000fa
:089ab400400020000000060044
:020000040000fa
:089abc0040002000000006003c
:020000040000fa
:089ac400308f88001cf607003a
:020000040000fa
:049acc000000060090
:020000040000fa
:049ad000000006008c
:020000040000fa
:049ad4000000060088
:020000040000fa
:049ad8000000060084
:020000040000fa
:020000040005f5
:045fe000ceff0000f0
:020000040000fa
:020000040005f5
:045fe400ffff0000bb
:020000040000fa
:020000040005f5
:045fe80060ff000056
:020000040000fa
:020000040005f5
:045fec0059ff000059
:020000040000fa
:020000040005f5
:045ff00038ff000076
:020000040000fa
:020000040005f5
:045ff400ffff0000ab
:00000001FF
